:020000040800F2
:1000000098220020850200080F410008B13A00083C
:10001000C5400008590E0008914C0008000000007F
:100020000000000000000000000000003143000854
:10003000C70F000800000000134100083343000808
:100040009F0200089F0200089F0200089F0200080C
:100050009F0200089F0200089F0200089F020008FC
:100060009F0200089F0200089F0200089F020008EC
:100070009F0200089F0200085D0E00086D0E000838
:100080009F0200087D0E00089F0200089F020008E2
:100090009F0200089F0200089F0200089F020008BC
:1000A0009F0200089F0200089F0200089F020008AC
:1000B0009F0200089F0200089F0200089F0200089C
:1000C0009F0200089F0200089F0200089F0200088C
:1000D0009F020008514C0008614C0008714C000858
:1000E0009F0200089F0200089F0200089F0200086C
:1000F0009F0200089F0200089F0200089F0200085C
:100100009F0200089F0200089F0200089F0200084B
:10011000714600089F0200080544000815440008C5
:100120008D0E00089F0200089F0200089F02000831
:100130009F0200089F0200089F0200089F0200081B
:100140009F0200089F0200089F0200089F0200080B
:100150009F0200089D0E0008AD0E0008814C0008AB
:100160009F0200089F0200089F0200089F020008EB
:100170009F0200089F0200089F0200080000000084
:100180009F0200089F02000800F002F800F06AF8E1
:100190000AA090E8000C82448344AAF10107DA45E2
:1001A00001D100F05FF8AFF2090EBAE80F0013F0CA
:1001B000010F18BFFB1A43F001031847F89E000017
:1001C000189F00000A444FF0000C10F8013B13F098
:1001D000070408BF10F8014B1D1108BF10F8015BA0
:1001E000641E05D010F8016B641E01F8016BF9D193
:1001F00013F0080F1EBF10F8014BAD1C0C1B09D1EA
:100200006D1E58BF01F801CBFAD505E014F8016B5B
:1002100001F8016B6D1EF9D59142D6D370470000ED
:100220000023002400250026103A28BF78C1FBD8FF
:10023000520728BF30C148BF0B607047642900F0E7
:100240005581782900F08E81632900F0128473298A
:1002500000F01784002070471FB509F0D9FE1FBDBC
:1002600010B510BD00F028FC1146FFF7F5FF07F0B0
:1002700051FA00F046FC03B4FFF7F2FF03BC04F0B0
:10028000C3FD00000948804709480047FEE7FEE734
:10029000FEE7FEE7FEE7FEE7FEE7FEE7FEE7FEE736
:1002A00004480549054A064B70470000F143000821
:1002B00089010008981C002098220020981E002028
:1002C000981E00207047704753EA020C00F06980C6
:1002D0002DE9F04B4FF00006002B1FBFB3FA83F55A
:1002E00003FA05F424FA05F65E4012BF1643B2FA8B
:1002F00082F502FA05F4C5F120051EBF22FA05FCBD
:1003000044EA0C04203556EA044C4FEA144418BF62
:10031000641C4FF000084FF00009904271EB030C91
:1003200039D3002919BFB1FA81F701FA07F6B0FAFB
:1003300080F700FA07F6C7F120071EBF20FA07FC76
:1003400046EA0C062037B6FBF4FCA7EB0507103F86
:1003500007F01F0BCBF120060CFA0BFB2CFA06F66C
:1003600044BFB3460026202FA4BF5E464FF0000BCB
:100370005BEA060C08BF4FF0010B19EB0B09ABFB56
:10038000027C48EB0608C01B06FB02CC0BFB03CC2F
:1003900071EB0C01C1E70B46024641464846BDE8F9
:1003A000F08B13B54FF000004FF00001AFF3008069
:1003B000BDE81C40704710B54C1084EA530404D5C6
:1003C0004042C1F1000138BF491E1B4204D55242D0
:1003D000C3F1000338BF5B1EFFF776FF14F0804FB8
:1003E00004D04042C1F1000138BF491E14F0004F53
:1003F00004D05242C3F1000338BF5B1E10BD0000A1
:100400000FB4044910B503AA029800F03FFB10BCDA
:100410005DF814FB100200200FB41CB50C0007AAF5
:10042000009001D02044401E074B7B446946019058
:10043000069800F0F4FA002C03D06946002000F082
:1004400001FB1CBC5DF814FB2106000070B50446DE
:1004500085690068C10601D5302600E02026C00766
:1004600007D070BDD4E9012130469047206A401C76
:1004700020626D1EF6D570BD70B5044685690078A2
:10048000C00707D170BDD4E9012120209047206A20
:10049000401C20626D1EF6D570BD70B50C46054639
:1004A000012A05D02878800600D5EA69002302E0F9
:1004B000012305E05B1C934202D2E05C0028F9D1E5
:1004C000A869E618C01AA861286A18442862284654
:1004D000FFF7BCFF04E0D5E9012114F8010B9047B8
:1004E000B442F8D32846FFF7C7FF70BD2DE9F041AD
:1004F0000646002410687529314616A510D0AFF3C2
:100500000080002802DA404213A507E031688A071C
:1005100001D512A502E0490704D511A5012401E087
:10052000AFF3008000210A2206F1240709E0B0FBA6
:10053000F2FCB0FBF2F302FB1C003030785418469A
:10054000491C0028F3D123462A463046BDE8F04135
:1005500000F007BA000000002D0000002B00000092
:100560002000000070B504460D4621461068AFF328
:1005700000802188090502D50F4A7A4402E00E4A1C
:100580007A440E32002104F1240305E000F00F0646
:100590000009965D5E54491C0028F7D1207800239D
:1005A000000704D5702D02D009B102231132204674
:1005B000BDE8704000F0D5B9FC9A00002DE9F05F6D
:1005C000894604464FF0000ADFF824B1FB44C0F826
:1005D00020A02046E168884700287DD0252806D045
:1005E000D4E901219047206A401C2062F1E70025F0
:1005F0005F462046E16888472028064607DB312E03
:1006000005D2B81910F8200C08B10543F1E7A80786
:1006100001D525F00405C4F81CA00027C4F818A0D3
:100620002A2E09D0304604F0E1FB38B304EB8708EA
:10063000303EC8F8186019E059F8041B204604EB56
:1006400087029161E1688847012F064618D1E06969
:10065000002820DA25F020051DE0D8F8180000EB6E
:10066000800006EB40003038C8F818002046E168EA
:100670008847064604F0BAFB0028EED1012F0AD0C5
:100680002E2E08D12046E16888477F1C0646022F9F
:1006900045F02005C4DBA069002803DA404245F09C
:1006A0000105A061E80701D025F01005A6B1A6F16B
:1006B0004100192802D8203645F400654A463146E3
:1006C000204625604D46FFF7B9FD60B1012807D0EF
:1006D000ED1D25F0070000E007E000F1080978E7CC
:1006E00005F1040975E730467AE7206ABDE8F09F16
:1006F000D29A000040EA010310B59B070FD1042AEB
:100700000DD310C808C9121F9C42F8D020BA19BADC
:10071000884201D9012010BD4FF0FF3010BD1AB141
:10072000D30703D0521C07E0002010BD10F8013B96
:1007300011F8014B1B1B07D110F8013B11F8014BBD
:100740001B1B01D1921EF1D1184610BD10B5431CE0
:1007500002E010F8011B71B18107FAD14FF00132AC
:1007600002C88C1A8C4314EAC211F9D0C01A0A06C6
:1007700003D0C01E10BDC01A10BD0A0401D0801ED7
:1007800010BD0902FCD0401E10BD40EA010370B547
:100790009B072ED14FF00136042A2AD308C810C96E
:1007A0009D1B9D43121F15EAC61517D0D8B2E1B2A2
:1007B000401A50EA056110D198B2A1B2401A50EA2D
:1007C00005410AD123F07F4024F07F41401A50EACE
:1007D000052102D1180EA0EB146070BDA342DBD03E
:1007E00018BA21BA884201D9012070BD4FF0FF30FC
:1007F00070BD0AB9002070BD10F8013B11F8014B23
:1008000063B1A3420AD1521E08D010F8013B11F87F
:10081000014B1BB1A34201D1521EEDD1181B70BD7B
:10082000032A40F2308010F0030C00F0158011F81C
:10083000013BBCF1020F624498BF11F801CB00F8F4
:10084000013B38BF11F8013BA2F1040298BF00F848
:1008500001CB38BF00F8013B11F0030300F0258005
:10086000083AC0F0088051F8043B083A51F804CB2C
:10087000A0E80810F5E7121D5CBF51F8043B40F8F2
:10088000043BAFF30080D20724BF11F8013B11F8FD
:1008900001CB48BF11F8012B24BF00F8013B00F841
:1008A00001CB48BF00F8012B704710B5203AC0F0CB
:1008B0000B80B1E81850203AA0E81850B1E8185061
:1008C000A0E81850BFF4F5AF5FEA027C24BFB1E89E
:1008D0001850A0E8185044BF18C918C0BDE810400F
:1008E0005FEA827C24BF51F8043B40F8043B08BF18
:1008F0007047D20728BF31F8023B48BF11F8012BDF
:1009000028BF20F8023B48BF00F8012B70474FF08A
:10091000000200B5134694469646203922BFA0E84F
:100920000C50A0E80C50B1F12001BFF4F7AF09075B
:1009300028BFA0E80C5048BF0CC05DF804EB89004C
:1009400028BF40F8042B08BF704748BF20F8022B8F
:1009500011F0804F18BF00F8012B704770477047A7
:1009600070472DE9F0470D4699469246044600F13E
:1009700024080168880604D5E06921F0100121608F
:1009800000E00120A84201DD471B00E00027A1692B
:100990007A1902EB0900081AA0612078C00602D477
:1009A0002046FFF753FD002608E0D4E901211AF89C
:1009B00006009047206A401C761C20624E45F4DBFE
:1009C0002078C0060AD52046FFF740FD06E0D4E9AE
:1009D000012130209047206A401C2062381EA7F178
:1009E0000107F4DC07E0D4E9012118F8050090477D
:1009F000206A401C2062281EA5F10105F3DC204678
:100A0000FFF73AFD2078000602D50220BDE8F08706
:100A10000120FBE701694A1C02610878704700B5B4
:100A20008FB0CDE901310021059105497944CDE927
:100A3000031011466846FFF7C1FD0FB000BD00006E
:100A4000E5FFFFFF0A6802F8010B0A607047D1E971
:100A500000239A4202D2531C0B601070704710B5ED
:100A6000436913B1AFF3008001E0FFF716FD0120E9
:100A700010BD127800F124010A7000224A70012290
:100A8000EDE711684FF0FF32E9E70000074B70B562
:100A90000D467B44FFF7C3FF0446284600F008F8E4
:100AA00010B14FF0FF3070BD204670BDB36A00003A
:100AB000007B00F080007047754600F029F8AE46D4
:100AC00005006946534620F00700854618B020B55A
:100AD000FFF7E6FBBDE820404FF000064FF00007AF
:100AE0004FF000084FF0000B21F00701AC46ACE8D6
:100AF000C009ACE8C009ACE8C009ACE8C0098D4643
:100B000070470446AFF300802046FFF7B4FB0000B7
:100B100000487047381C002055494A6822F440328A
:100B20004A604A6843681A434A600268526822F47D
:100B3000807203685A6002685368026943EA0222BD
:100B400003685A600268526822F0407203685A6073
:100B50000268526883681A4303685A6002689268A0
:100B600022F4006203689A6002689268C3681A43BC
:100B700003689A603F4B826A9A4218D00268926872
:100B800022F0706203689A6002689268836A1A436E
:100B900003689A600268926822F0405203689A6083
:100BA00002689268C36A1A4303689A600BE002689D
:100BB000926822F0706203689A600268926822F07C
:100BC000405203689A600268926822F00202036849
:100BD0009A6002689368027E43EA420203689A6060
:100BE0002022125CA2B10268526842F400620368DB
:100BF0005A600268526822F4604203685A600268D0
:100C00005368426A521E43EA423203685A6005E062
:100C10000268526822F4006203685A600268D26A6D
:100C200022F470020368DA620268D36A828B521E71
:100C300043EA02520368DA620268926822F40072A0
:100C400003689A600268936890F8302043EA422271
:100C500003689A600268926822F4806203689A606E
:100C600002689368426943EA822203689A60704787
:100C7000002301400100000F30B52DED028B81B043
:100C8000044614E05A480068401C59490860084668
:100C900000684FF6FF71884209DB00205449086064
:100CA000544890ED000B01B0BDEC028B30BD20210B
:100CB000514800F015FF0028E4D1082C2DD2DFE8C0
:100CC00004F004090E13181D22270821012000F04A
:100CD0009DF822E01821012000F098F81DE028215D
:100CE000012000F093F818E03821012000F08EF880
:100CF00013E04821012000F089F80EE0582101207E
:100D000000F084F809E06821012000F07FF804E099
:100D10007821012000F07AF800BF00BF00221021E6
:100D2000354800F0EFFEFC25284604F045FD00257F
:100D3000284604F041FD0125284604F03DFD05202C
:100D400006F0EAF904F00AFD8DF8000004F006FD53
:100D50008DF8010004F002FD8DF802009DF80000FE
:100D600000049DF8011040EA01209DF8021008439C
:100D700022490860052006F0CFF920480068204984
:100D800008600846006800F40000F8B108460068F2
:100D9000C043086008460068C0F3160008600846B3
:100DA0000068401C08600846006840420860084629
:100DB000006808F02EFF41EC180B9FED120B53EC6E
:100DC000102B08F03DFF0B4A03C20DE00C480068F1
:100DD00008F01FFF41EC180B9FED0A0B53EC102B92
:100DE00008F02EFF034A03C2024890ED000B5AE7B9
:100DF00040000020380000200004024030000020A5
:100E00003400002085F90F270088433F70B5044661
:100E10000D46002210210F4800F074FE00BF202173
:100E20000C4800F05DFE0028F9D104F00F0040F0FE
:100E30005006304604F0C0FC0026304604F0BCFCEE
:100E4000284604F0B9FC00221021024800F05AFEA6
:100E500070BD00000004024000BFFEE710B502486C
:100E600000F050FB10BD0000C806002010B502487D
:100E700000F048FB10BD0000A805002010B5024896
:100E800000F040FB10BD00006806002010B50248CD
:100E900000F038FB10BD00005C02002010B50248D5
:100EA00000F030FB10BD00002807002010B50248FC
:100EB00000F028FB10BD000008060020014608785D
:100EC00010381823B0FBF3F20848805CC865032A89
:100ED00005D908686FF30900001D886503E00868FC
:100EE0006FF309008865886D7047000024A0000832
:100EF000014600208A6A8B69CBB932B1012A0DD034
:100F0000022A03D0032A10D10EE000BFCB6A03F0FF
:100F10008073B3F1807F00D1012007E0CB6AB3F189
:100F2000C07F00D1012001E000E000BF34E08B6908
:100F3000B3F5005F1AD132B1012A07D0022A03D0DB
:100F4000032A11D10AE000BF01200EE0CB6A03F0B2
:100F50008073B3F1807F00D1012006E0CB6AB3F14A
:100F6000C07F00D1012000E000BF15E032B1012AAE
:100F700005D0022A04D0032A0CD103E000BF00BF31
:100F8000012008E0CB6A03F08073B3F1807F00D1C9
:100F9000012000E000BF00BF704730B5046824683E
:100FA00024F4802405682C60046863608468402C05
:100FB00004D10468A2600468E16003E00468A160F1
:100FC0000468E26030BD704772B600BFFEE7000003
:100FD00001460846024B33F8100002B290B2704747
:100FE000CE00002001460846024B33F8100002B242
:100FF00090B27047D608002030B5A0F11002D41787
:1010000002EB5474E410094D2B5DD41702EB5474B9
:10101000E410A2EBC4050124AC401C4014B1012231
:101020000A7001E000220A7030BD0000C0080020F4
:1010300030B50246D41702EB5474E410094D2B5D11
:101040000246D41702EB5474E410A2EBC405012449
:10105000AC401C4014B101220A7001E000220A7069
:1010600030BD0000CA08002038B5024600200090BC
:1010700000BF92F83C00012801D1022038BD0120B8
:1010800082F83C0000BF0868092816D91068C068BB
:101090000C780A3C04EB44050724AC40A0431468D8
:1010A000E0600C780A3C04EB44048868A0401468B3
:1010B000E46820431468E06013E0106800690C786D
:1010C00004EB44050724AC40A043146820610C786D
:1010D00004EB44048868A040146824692043146821
:1010E00020614868072817D21068406B0C79641E8D
:1010F00004EB84051F24AC40A04314686063088897
:1011000080B20C79641E04EB8404A0401468646B04
:1011100020431468606331E048680D2817D21068D6
:10112000006B0C79E41F04EB84051F24AC40A04342
:1011300014682063088880B20C79E41F04EB8404EF
:10114000A0401468246B20431468206316E01068E4
:10115000C06A0C790D3C04EB84051F24AC40A0430D
:101160001468E062088880B20C790D3C04EB8404BA
:10117000A0401468E46A20431468E062194B1A4CDA
:101180001068A04206D10868122803D1586840F4BC
:1011900080005860144C1068A0421CD108681028C8
:1011A00002D00868112816D1586840F40000586031
:1011B000086810280FD10D4800680D4CB0FBF4F002
:1011C00000EB80004000009002E00098401E00907C
:1011D00000980028F9D100BF002082F83C0000BF31
:1011E00000BF4BE700230140002001402800002001
:1011F00040420F0001460868C06C704770B5044655
:1012000000250CB9012070BD1549A06A884200D0A4
:1012100000BF206C30B9204600F024F80020606444
:1012200084F83C00206C00F0100088B9206C20F499
:10123000885040F0020020642046FFF76DFC00203B
:101240006064206C20F0020040F00100206400E0A7
:10125000012500BF002084F83C0000BF2846D2E7EB
:101260000100000F10B586B00446142101A8FFF755
:101270004EFB1949206888422BD100BF0020009006
:101280001648006840F480701449086008460068F9
:1012900000F48070009000BF00BF00BF00200090ED
:1012A0000E481438006840F004000C4914390860F6
:1012B0000846006800F00400009000BF00BF012055
:1012C0000190032002900020039001A9044800F03F
:1012D0000DFB06B010BD0000002001404438024064
:1012E0000008024008B501460020009000BF91F8B8
:1012F0003C00012801D1022008BD012081F83C00FA
:1013000000BF0868806800F00100A0B90868806824
:1013100040F001000B6898603F4800683F4BB0FB0D
:10132000F3F000EB4000009002E00098401E0090B7
:1013300000980028F9D10868806800F001000028B2
:1013400060D0086C40F20163984340F480700864F8
:101350000868406800F4806028B1086C20F40050F0
:1013600040F480500864086C00F48050B0F5805F51
:1013700004D1486C20F00600486401E00020486475
:1013800000BF002081F83C0000BF254A6FF022001A
:101390000B681860506800F01F0018BB214B0868EC
:1013A000984213D0204B0868984204D1101D006861
:1013B00000F01F0050B11D4B086898422AD1184810
:1013C000001D006800F01F00102823D20868806804
:1013D00000F04050F0B90868806840F080400B6829
:1013E000986017E00F4B0868984213D1086880682E
:1013F00000F0405070B90868806840F080400B6889
:10140000986007E0086C40F010000864486C40F0F9
:101410000100486400206FE72800002040420F00D0
:101420000023014000200140002101400022014032
:1014300070B50446A56D00F06BFB064694F83500C8
:10144000022808D08020606500BF002084F83400A6
:1014500000BF012070BD2068006820F016002168E0
:1014600008602068406920F0800021684861206C95
:1014700008B9A06C28B12068006820F00800216835
:1014800008602068006820F001002168086010E012
:1014900000F03EFB801B05280BD92020606503204F
:1014A00084F8350000BF002084F8340000BF03201A
:1014B000D0E72068006800F001000028E8D194F827
:1014C0005C103F208840A860012084F8350000BFF0
:1014D000002084F8340000BF00BFBBE7014691F84C
:1014E0003500022803D08020486501207047052080
:1014F00081F835000868006820F001000A68106073
:101500000020F3E7F8B50446002000908C480068FE
:101510004FF41651B0FBF1F7A56D2E6894F85C10EE
:1015200008208840304098B12068006800F004002E
:1015300070B12068006820F004002168086094F809
:101540005C1008208840A860606D40F00100606574
:1015500094F85C1001208840304068B120684069F0
:1015600000F0800040B194F85C1001208840A86031
:10157000606D40F00200606594F85C1004208840C3
:10158000304068B12068006800F0020040B194F873
:101590005C1004208840A860606D40F00400606525
:1015A00094F85C1010208840304078B320680068C0
:1015B00000F0080050B394F85C1010208840A86038
:1015C0002068006800F4802080B12068006800F482
:1015D000002028B9206CC8B12046216C884715E04E
:1015E000A06C98B12046A16C88470FE02068006885
:1015F00000F4807028B92068006820F00800216895
:101600000860206C10B12046216C884794F85C106B
:10161000202088403040002865D02068006800F015
:10162000100000285FD094F85C1020208840A8604B
:1016300094F83500052828D12068006820F01600AD
:10164000216808602068406920F0800021684861B6
:10165000206C08B9A06C28B12068006820F0080050
:101660002168086094F85C103F208840A860012041
:1016700084F8350000BF002084F8340000BF206DDE
:1016800010B12046216D8847F8BD2068006800F43D
:10169000802080B12068006800F4002028B9606CC8
:1016A00010B12046616C88471DE0E06BD8B1204640
:1016B000E16B884717E02068006800F4807068B923
:1016C0002068006820F0100021680860012084F87C
:1016D000350000BF002084F8340000BFE06B10B17B
:1016E0002046E16B8847606D38B3606D00F0010003
:1016F000F0B1052084F835002068006820F0010072
:101700002168086000BF0098401C0090B84200D9D2
:1017100005E02068006800F001000028F3D100BF58
:10172000012084F8350000BF002084F8340000BF99
:10173000E06C10B12046E16C884700BFA4E70000D0
:10174000280000202DE9F0410446002500F0E0F9D2
:10175000074614B90120BDE8F081606A00B100BFFE
:10176000022084F8350000BF002084F8340000BF58
:101770002068006820F00100216808600AE000F09D
:10178000C7F9C01B052805D920206065032084F80F
:101790003500E0E72068006800F001000028EED185
:1017A0002068056821480540D4E901010843E16843
:1017B00008432169084361690843A1690843E16955
:1017C0000843216A08430543606A042803D1D4E929
:1017D0000B0108430543206805602068456925F032
:1017E0000705606A0543606A04280DD1A06A0543B5
:1017F000E06A48B12046FFF77BFB28B140206065D6
:10180000012084F83500A6E7206845612046FFF7EF
:1018100055FB064694F85C103F208840B0600020DD
:101820006065012084F83500002094E73F8010F0C7
:101830002DE9F04704460D4616461F464FF00008B6
:10184000D4F8589000BF94F83400012802D1022047
:10185000BDE8F087012084F8340000BF94F835001B
:10186000012825D1022084F83500002060653B4620
:10187000324629462046FFF790FB94F85C103F2043
:101880008840C9F808002068006840F01600216808
:101890000860206C28B12068006840F008002168CA
:1018A00008602068006840F001002168086006E0D8
:1018B00000BF002084F8340000BF4FF0020840460B
:1018C000C6E7000070B5044600F022F9064625463A
:1018D000681C10B104480078054400BF00F018F9F6
:1018E000801BA842FAD370BD24000020F8B5024640
:1018F0000B460025002400200021D6E0012606FA30
:1019000001F51E6806EA0504AC4274D11E7906F0A2
:101910000306012E04D01E7906F00306022E13D111
:1019200090684F000326BE40B0434F00DE68BE40C3
:1019300030439060506801268E40B0431E79C6F354
:1019400000168E40304350601E7906F00306032EC9
:1019500009D0D0684F000326BE40B0434F009E68B8
:10196000BE403043D0601E7906F00306022E13D12C
:10197000CF0802F1200656F827004E07F70E0F2673
:10198000BE40B0434F07FF0E1E69BE403043CF0834
:1019900002F1200646F8270010684F000326BE40DB
:1019A000B0431E7906F003064F00BE40304310607E
:1019B0005E6806F44036002E76D000BF0026009602
:1019C0003C4E366846F480463A4F3E603E463668A6
:1019D00006F48046009600BF00BF374E8F0856F8C9
:1019E00027008E07370F0F26BE40B043334EB2425A
:1019F00002D1002624E057E0314EB24201D1012647
:101A00001EE0304EB24201D1022619E02E4EB24203
:101A100001D1032614E02D4EB24201D104260FE07D
:101A20002B4EB24201D105260AE02A4EB24201D124
:101A3000062605E0284EB24201D1072600E008261E
:101A40008F073F0FBE4030431B4E8F0846F82700DC
:101A5000224E3068A0435E6806F4801606B120432B
:101A60001E4E3060361D3068A0435E6806F40016D6
:101A700006B12043194E361D3060184E361F3068AF
:101A8000A0435E6806F4003606B12043134E361FAD
:101A90003060361F3068A0435E6806F4803606B1B9
:101AA00020430E4E083E3060491C1029FFF426AF3B
:101AB000F8BD0000443802400838014000000240F0
:101AC0000004024000080240000C024000100240E6
:101AD0000014024000180240001C0240083C014073
:101AE000024613690B400BB1012000E00020704753
:101AF00010B5426921EA020302EA010443EA044301
:101B0000836110BD0AB1816101E00B0483617047FC
:101B100001480068704700001C00002070B50446B2
:101B20000CB9012070BD94F83D0028B9002084F85C
:101B30003C00204600F0DAF8242084F83D002068BC
:101B4000006820F00100216808602068006840F407
:101B50000040216808602068006820F40040216887
:101B6000086000F0ADFA05465C496068884206D816
:101B70005B48854201D2012007E0002005E059487A
:101B8000854201D2012000E00020012800D1C9E7F0
:101B90005548B5FBF0F62068406820F03F00304320
:101BA000216848604D496068884201D8701C07E090
:101BB0004FF4967070434FF47A71B0FBF1F0401C13
:101BC0002168096A21F03F010843216808624349FE
:101BD0006068884214D8681E61684900B0FBF1F063
:101BE000401CC0F30B00042801D204203DE0681E15
:101BF00061684900B0FBF1F0401CC0F30B0034E019
:101C0000A06838B9681E616801EB4101B0FBF1F0D2
:101C1000401C0AE0681E616801EBC10202EB011181
:101C2000B0FBF1F0401C40F48040C0F30B0008B959
:101C300001201AE0A06848B9681E616801EB410103
:101C4000B0FBF1F0401CC0F30B000CE0681E6168B3
:101C500001EBC10202EB0111B0FBF1F0401CC0F33B
:101C60000B0040F4804040F400402168C9694CF604
:101C7000FF72914308432168C861D4E90701084312
:101C80002168096821F0C001084321680860D4E98F
:101C9000031008432168896848F2FF3291430843E2
:101CA00021688860D4E9050108432168C96821F0EA
:101CB000FF0108432168C8602068006840F0010007
:101CC0002168086000202064202084F83D00002066
:101CD000206384F83E0000BF24E70000A0860100D6
:101CE00080841E0000093D0040420F0010B586B000
:101CF0000446142101A8FEF70AFE1B492068884209
:101D00002FD100BF002000901848006840F002006A
:101D1000164908600846006800F00200009000BF05
:101D200000BFC020019012200290002003900320E9
:101D300004900420059001A90D48FFF7D7FD00BFCE
:101D40000020009009481030006840F40010074956
:101D5000103108600846006800F40010009000BFD1
:101D600000BF06B010BD00000054004030380240F3
:101D70000004024003480068034909780844014907
:101D8000086070471C0000202400002010B50D489A
:101D9000006840F400700B4908600846006840F491
:101DA000806008600846006840F480700860032086
:101DB00000F0AAF8032000F007F800F02BF800204C
:101DC00010BD0000003C024070B504460E4800788B
:101DD0004FF47A71B1FBF0F00C490968B1FBF0F5F2
:101DE000284600F0FBFD08B1012070BD102C07D281
:101DF00000222146501E00F049F80548046001E029
:101E00000120F2E70020F0E7240000202800002055
:101E10002000002008B500BF002000901048006896
:101E200040F480400E4908600846006800F4804095
:101E3000009000BF00BF00BF00200090081F006896
:101E400040F08050091F08600846006800F080508C
:101E5000009000BF00BF052000F056F808BD00004C
:101E6000443802400146084600280DDB00BF00BF91
:101E700000F01F0301229A4043099B0003F1E02375
:101E8000C3F8002100BF00BF00BF70472DE9F05F1D
:101E900080460D461646002702F08CFF074639465D
:101EA0002A46334601F00700C0F1070ABAF1040FD1
:101EB00002D94FF0040A01E0C0F1070AD14600F14F
:101EC000040ABAF1070F02D24FF0000A01E0A0F1B4
:101ED000030AD4464FF0010A0AFA09FAAAF1010AE4
:101EE0000AEA020A0AFA0CFA4FF0010B0BFA0CFB91
:101EF000ABF1010B0BEA030B4AEA0B042146404607
:101F000002F060FFBDE8F09F00BF00F00702064B43
:101F100019684FF6FF031940044B0B4343EA0221B3
:101F2000014B196000BF70470CED00E00000FA059E
:101F300070B504460D460CB9012070BD58480068C4
:101F400000F00700A84209D255490D700846006804
:101F500000F00700A84201D00120EEE7207800F051
:101F6000020002281DD1207800F00400042805D1C9
:101F70004C48006840F4E0504A490860207800F07E
:101F80000800082805D14748006840F460404549EA
:101F900008604448006820F0F000A1680843414907
:101FA0000860207800F00100A8B36068012807D11C
:101FB0003C4808380068C0F34040B8B90120BCE78D
:101FC0006068022802D06068032807D135480838C5
:101FD0000068C0F3406048B90120AEE731480838D6
:101FE0000068C0F3400008B90120A6E72D4800684A
:101FF00020F00300616808432A490860FFF788FD64
:10200000064609E0FFF784FD801B41F288318842D3
:1020100002D9032091E707E02248006800F00C0095
:102020006168B0EB810FEDD11D48006800F007003A
:10203000A84209D91A490D700846006800F0070047
:10204000A84201D0012078E7207800F0040004289D
:1020500007D11448006820F4E050E16808431149B2
:102060000860207800F00800082808D10D480068B2
:1020700020F46040216940EAC1000A49086000F08C
:102080003FF808490968C1F30311074A515CC84089
:102090000649086006480068FFF796FE00204CE7F6
:1020A000003C0240083802402CA000082800002014
:1020B0002000002001480068704700002800002030
:1020C00000B5FFF7F7FF04490968C1F38221034A0D
:1020D000515CC84000BD0000083802403CA0000828
:1020E00000B5FFF7E7FF04490968C1F34231034A2D
:1020F000515CC84000BD0000083802403CA0000808
:102100002DE9F047002400250026A1462548006857
:1021100000F00C0020B1042805D008283AD105E0D1
:10212000DFF8849039E0DFF8849036E01D48001F26
:10213000006800F03F041B48001F006800F48000A6
:1021400078B11A481749091F0968C1F38811A0FB23
:1021500001700146224600233846FEF7B5F80546D1
:102160000EE011480F49091F0968C1F38811A0FB4F
:1021700001700146224600233846FEF7A5F80546C1
:102180000848001F0068C0F30140401C4600B5FB32
:10219000F6F902E0DFF8109000BF00BF4846BDE846
:1021A000F0870000083802400024F40000127A0092
:1021B000F8B504460CB90120F8BD207800F0010004
:1021C000002874D0F948006800F00C0004280DD0F5
:1021D000F648006800F00C00082813D1F348001FEF
:1021E000006800F48000B0F5800F0BD1EF4808388C
:1021F0000068C0F34040002859D06068002856D1DC
:102200000120D9E700BF6068B0F5803F08D1E748FA
:102210000838006840F48030E449083908601EE05E
:102220006068B0F5A02F0DD1E0480838006840F490
:102230008020DE49083908600846006840F4803094
:1022400008600CE0D9480838006820F48030D7498D
:10225000083908600846006820F48020086000BF44
:10226000606890B1FFF754FC054606E0FFF750FCAC
:10227000401B642801D903209EE7CC480838006839
:10228000C0F340400028F1D011E0FFF741FC0546C3
:1022900006E0FFF73DFC401B642801D903208BE7D3
:1022A000C24808380068C0F340400028F1D12078C7
:1022B00000F0020002285FD1BC48006800F00C006A
:1022C00058B1BA48006800F00C0008281CD1B74883
:1022D000001F006800F48000B0B9B44808380068F6
:1022E000C0F3400020B1E068012801D0012063E77D
:1022F000AE480838006820F0F800216940EAC100C3
:10230000AA490839086037E0E06800B30120A8490D
:102310000860FFF7FDFB054606E0FFF7F9FB401BF1
:10232000022801D9032047E7A04808380068C0F315
:1023300040000028F1D09D480838006820F0F800DF
:10234000216940EAC10099490839086014E0002079
:1023500097490860FFF7DCFB054606E0FFF7D8FB6E
:10236000401B022801D9032026E79048083800685E
:10237000C0F340000028F1D1207800F008000828C0
:102380002CD16069A8B101208A490860FFF7C0FB21
:10239000054606E0FFF7BCFB401B022801D90320DD
:1023A0000AE782486C300068C0F340000028F1D092
:1023B00014E000207F490860FFF7AAFB054606E00D
:1023C000FFF7A6FB401B022801D90320F4E677485B
:1023D0006C300068C0F340000028F1D1207800F094
:1023E0000400042870D1002770483830006800F0DD
:1023F000805090B900BF002000906C4838300068D1
:1024000040F080506949383108600846006800F0A3
:102410008050009000BF00BF01276748006800F4AB
:102420008070B0B96448006840F480706249086008
:10243000FFF76EFB054606E0FFF76AFB401B02282C
:1024400001D90320B8E65C48006800F480700028D9
:10245000F2D000BFA068012808D154486830006855
:1024600040F001005149683108601DE0A06805286E
:102470000DD14E486830006840F004004B49683187
:1024800008600846006840F0010008600CE047481A
:102490006830006820F0010044496831086008464F
:1024A000006820F00400086000BFA068A8B1FFF732
:1024B0002FFB054609E0FFF72BFB401B41F288315B
:1024C000884202D9032077E626E038486830006861
:1024D000C0F340000028EED013E0FFF719FB0546DB
:1024E00008E0FFF715FB401B41F28831884201D913
:1024F000032061E62D4868300068C0F340000028E2
:10250000EFD1012F07D129483830006820F08050E2
:1025100026493831086000BFA069002845D023480B
:10252000006800F00C0008285DD0A069022845D1A1
:1025300000201F490866FFF7EBFA054606E0FFF7A3
:10254000E7FA401B022801D9032035E6174808386E
:102550000068C0F340600028F1D1D4E907010843C6
:10256000616A40EA81110122A06AC2EB500041EA8F
:1025700000412C20005D41EA00600C49091F086001
:1025800001200B490866FFF7C3FA054606E0FFF78E
:10259000BFFA401B022801D903200DE60348083882
:1025A0000068C0F340600028F1D049E008380240DC
:1025B00000004742800E4742007000400020214941
:1025C0000866FFF7A5FA054606E0FFF7A1FA401BEB
:1025D000022801D90320EFE51B480068C0F34060E2
:1025E0000028F2D12CE0A069012800D1E4E51648CA
:1025F000001D0668A069012820D006F48001E0696A
:1026000081421BD106F03F01206A814216D147F674
:10261000C0703040616AB0EB811F0FD106F44031C9
:102620000122A06AC2EB5000B1EB004F06D106F0C8
:1026300070612C20005DB1EB006F01D00120BBE583
:102640000020B9E5000047420038024010B50446BA
:102650000CB9012010BD606A38B96068B0F5827F9E
:1026600000D105E00021E16102E00021216161610A
:102670000021A16294F8510028B9002084F850008C
:10268000204600F047F8022084F8510020680068D6
:1026900020F0400021680860A08800F48270218941
:1026A00001F404410843A18901F400610843217C3D
:1026B00001F002010843217D01F001010843218B53
:1026C00001F400710843217F01F038010843202103
:1026D000095D01F080010843218D01F40051084398
:1026E000216808600421A06901EA104094F82410D0
:1026F00001F010010843216848602068C06920F497
:1027000000602168C86100206065012084F85100E4
:1027100000209FE710B586B00446142101A8FEF7FB
:10272000F6F81B492068884230D100BF0020009095
:102730001848006840F48040164908600846006860
:1027400000F48040009000BF00BF00BF0020009058
:1027500010481038006840F002000E491039086037
:102760000846006800F00200009000BF00BF4FF470
:1027700070400190022002900020039003200490FA
:102780000520059001A90448FFF7B0F806B010BD78
:102790000038004040380240000402402DE9FF5F4D
:1027A0000446884691461D460E9E01200290002058
:1027B000019000BF94F85000012803D1022004B01A
:1027C000BDE8F09F012084F8500000BFFFF7A0F99A
:1027D000074694F851B060680390AA46BBF1010F18
:1027E0000BD00398B0F5827F04D1A06810B9BBF17B
:1027F000040F02D002200190E9E0B8F1000F03D0ED
:10280000B9F1000F00D015B901200190DFE094F874
:102810005100042802D0052084F851000020606592
:10282000C4F83890E587A587C4F83080E586A5868A
:10283000206460642068006800F04000402805D0F3
:102840002068006840F0400021680860E068B0F54A
:10285000006F4DD1606810B1BAF1010F09D1206B42
:1028600000882168C860206B801C2063E08E401EB9
:10287000E08636E02068806800F00200022810D16F
:10288000E08E70B1029801280BD1206B008821687E
:10289000C860206B801C2063E08E401EE086002014
:1028A00002902068806800F0010068B1E08F58B1A4
:1028B0002068C068A16B0880A06B801CA063E08FBB
:1028C000401EE08701200290FFF722F9C01BB042B2
:1028D00007D3701C28B103200190012084F8510017
:1028E00075E0E08E0028C5D1E08F0028C2D14DE010
:1028F000606810B1BAF1010F09D1206B007821682E
:102900000873206B401C2063E08E401EE08637E099
:102910002068806800F00200022810D1E08E70B1BB
:10292000029801280BD1206B007821680873206B76
:10293000401C2063E08E401EE0860020029020684C
:10294000806800F0010068B1E08F58B12068C0686D
:10295000A16B0870A06B401CA063E08F401EE08755
:1029600001200290FFF7D4F8C01BB04201D3701CC5
:1029700000B92EB903200190012084F8510026E00F
:10298000E08E0028C4D1E08F0028C1D13A463146FC
:10299000204601F0BFFB20B101200190202060659E
:1029A00015E0A06850B900BF002000902068C06802
:1029B000009020688068009000BF00BF606D10B17B
:1029C0000120019002E0012084F8510000BF00BF07
:1029D000002084F8500000BF0198F0E670B504466E
:1029E0002546681EB0F1807F01D301200FE0681EEC
:1029F0004FF0E02148610F214FF0FF3002F0E2F983
:102A000000204FF0E021886107200861002070BDA0
:102A10007047704730B502460B4600BF92F83C0045
:102A2000012801D1022030BD012082F83C0000BF06
:102A3000022082F83D00106844681068816824F024
:102A400070041868044310684460184D1068A84268
:102A50001BD01068B0F1804F17D0154D1068A842F8
:102A600013D0144D1068A8420FD0134D1068A8421F
:102A70000BD0124D1068A84207D0114D1068A84223
:102A800003D0104D1068A84205D121F0800158688C
:102A9000014310688160012082F83D0000BF0020E2
:102AA00082F83C0000BF00BFBDE70000000001400D
:102AB0000004004000080040000C004000040140F9
:102AC000004001400018004010B504460CB9012038
:102AD00010BD94F83D0028B9002084F83C00204641
:102AE00000F026F8022084F83D00211D206801F046
:102AF00099FC012084F8460000BF84F83E000121C3
:102B00003F200155402001554120015500BF00BF25
:102B1000012084F8420043200155442001554520FE
:102B2000015500BF012084F83D000020D0E70000DF
:102B300038B504461C492068884218D100BF0020DF
:102B400000901A48006840F01000184908600846D4
:102B5000006800F01000009000BF00BF0022114686
:102B60003620FFF793F93620FFF77CF91BE0104978
:102B70002068884217D100BF002000900B480068F1
:102B800040F02000094908600846006800F0200075
:102B9000009000BF00BF002201213720FFF776F927
:102BA0003720FFF75FF938BD001000404038024081
:102BB00000140040014691F83D00012801D0012099
:102BC0007047022081F83D000868C06840F00100AD
:102BD0000B68D8601A4B086898421BD00868B0F19F
:102BE000804F17D0174B0868984213D0164B0868CF
:102BF00098420FD0154B086898420BD0144B0868C8
:102C0000984207D0134B0868984203D0124B0868CB
:102C100098420CD10868806800F00702062A0CD0A0
:102C20000868006840F001000B68186005E008685B
:102C3000006840F001000B6818600020C0E7000049
:102C4000000001400004004000080040000C00406B
:102C5000000401400040014000180040014608689F
:102C6000C06820F001000A68D06000BF0868006AF0
:102C700041F21112104050B90868006A92101040D9
:102C800028B90868006820F001000A68106000BFD9
:102C9000012081F83D00002070472DE9F0410446F5
:102CA0000D4614B90120BDE8F08194F83D0028B923
:102CB000002084F83C00204600F053F8022084F8FD
:102CC0003D002068806844F20701884321688860DD
:102CD000211D206801F0A6FB2068D0F8088020683C
:102CE00086692068076A286840EA080840F20330CD
:102CF0008643A969A86840EA0120064340F60C40D3
:102D000086434FF2F0008643E969E86840EA012013
:102D1000064328690001296A40EA0130064327F08A
:102D2000220727F088076969686840EA01100743AD
:102D30002068C0F80880206886612068076201204A
:102D400084F8460084F83E0001213F20015501200F
:102D500084F8420043200155012084F83D00002002
:102D6000A1E770472DE9F04304460D4694F83E6014
:102D70003F20075D94F84280432010F804906DB91D
:102D8000012E02D1B8F1010F02D00120BDE8F0837D
:102D9000022084F83E0084F8420025E0042D0CD186
:102DA000012F02D1B9F1010F01D00120EEE702217C
:102DB0003F2001554320015516E0012E07D1012F78
:102DC00005D1B8F1010F02D1B9F1010F01D00120F5
:102DD000DCE7022084F83E0002213F20015502205A
:102DE00084F842004320015515B1042D0CD105E0B3
:102DF00001220021206801F089FB10E0012204215A
:102E0000206801F083FB0AE001220021206801F024
:102E10007DFB01220421206801F078FB00BF00BF88
:102E20002068006840F00100216808600020ADE7DC
:102E300070472DE9F04104460D461646002700BFB5
:102E400094F83C00012802D10220BDE8F081012065
:102E500084F83C0000BF96B9EB68D5E90012206801
:102E600001F066FB2068806920F00C002168886111
:102E700020688069A96808432168886141E0042EC0
:102E800013D1EB68D5E90012206801F099FB2068A6
:102E9000806920F440602168886120688069A968A1
:102EA00040EA0120216888612BE0082E12D1EB68EE
:102EB000D5E90012206801F0A0FB2068C06920F06D
:102EC0000C002168C8612068C069A96808432168AE
:102ED000C86116E00C2E13D1EB68D5E9001220680A
:102EE00001F0A7FB2068C06920F440602168C86138
:102EF0002068C069A96840EA01202168C86100E033
:102F0000012700BF002084F83C0000BF38469CE742
:102F100010B504460CB9012010BD94F83D0028B945
:102F2000002084F83C00204600F026F8022084F8B7
:102F30003D00211D206801F075FA012084F846004B
:102F400000BF84F83E0001213F200155402001557B
:102F50004120015500BF00BF012084F842004320FA
:102F60000155442001554520015500BF012084F83A
:102F70003D000020D0E7000010B586B004461421C3
:102F800001A8FDF7C4FC1B49206888422FD100BF6F
:102F9000002000901848006840F0010016490860C1
:102FA0000846006800F00100009000BF00BF00BFAD
:102FB0000020009010481438006840F010000E49BE
:102FC000143908600846006800F01000009000BF47
:102FD00000BF4FF42850019002200290002003907F
:102FE00004900120059001A90448FEF77FFC06B07B
:102FF00010BD0000000001404438024000100240B3
:1030000070B504462068C5682068066906F00200AD
:10301000022819D105F00200022815D1401F2168AD
:103020000861012020772068806900F0030018B152
:103030002046FFF7FDFE05E0204600F097F8204609
:1030400000F095F80020207706F00400042819D13C
:1030500005F00400042815D1C0432168086102204E
:1030600020772068806900F4407018B12046FFF78F
:10307000DFFE05E0204600F079F8204600F077F802
:103080000020207706F00800082819D105F0080074
:10309000082815D1C04321680861042020772068E2
:1030A000C06900F0030018B12046FFF7C1FE05E03B
:1030B000204600F05BF8204600F059F80020207709
:1030C00006F01000102819D105F01000102815D1B5
:1030D000C04321680861082020772068C06900F497
:1030E000407018B12046FFF7A3FE05E0204600F02F
:1030F0003DF8204600F03BF80020207706F0010064
:1031000048B105F0010030B16FF00100216808619D
:10311000204600F02DF806F08000802809D105F047
:103120008000802805D1C043216808612046FFF750
:103130006FFC06F04000402809D105F0400040280F
:1031400005D1C04321680861204600F033F806F03D
:103150002000202809D105F02000202805D1C043F7
:10316000216808612046FFF754FC70BD7047704726
:1031700010B504460C48844201D105F0DDFB0B4834
:1031800084420FD16FF001000849096808610748BF
:10319000FFF764FD064880880549C88000208880C4
:1031A00004F06EFD10BD0000B0030020F803002005
:1031B000241C002070477047704700002DE9F84F2D
:1031C0000446206805682068C668206847694FF093
:1031D0000009CA4605F00F09B9F1000F0AD105F040
:1031E000200038B106F0200020B1204601F006FB97
:1031F000BDE8F88FB9F1000F7CD007F0010018B9D5
:1032000006F49070002875D005F0010030B106F486
:10321000807018B1606C40F00100606405F004003B
:1032200030B107F0010018B1606C40F0020060643A
:1032300005F0020030B107F0010018B1606C40F0F9
:103240000400606405F0080048B106F0200010B9E1
:1032500007F0010018B1606C40F008006064606C19
:10326000002846D005F0200028B106F0200010B15B
:10327000204601F0C3FA20684069C0F3801A606CF0
:1032800000F0080010B9BAF1000F2DD0204601F06F
:103290005CFA2068406900F04000402820D100BF5F
:1032A00000BF2168143151E8001F21F0400021685F
:1032B000143141E80002002AF3D100BFE06B50B1A5
:1032C0007748E16B0865E06BFEF708F988B1E06BC1
:1032D000016D88470DE02046FFF76EFF09E009E029
:1032E0002046FFF769FF04E02046FFF765FF002056
:1032F00060647DE7206B012878D105F0100000287C
:1033000074D006F010000028FAD000BF0020009012
:1033100020680068009020684068009000BF00BFEF
:103320002068406900F04000402860D1E06B0068F0
:1033300040681FFA80F8B8F1000F56D0A08D4045C4
:1033400053DDA4F82E80E06BC069B0F5807F43D0D8
:1033500000BF00BF21680C3151E8001F21F48070CC
:1033600021680C3141E80002002AF3D100BF00BF00
:1033700000BF2168143151E8001F21F001002168CD
:10338000143141E80002002AF3D100BF00BF00BFA2
:103390002168143151E8001F21F0400021681431E8
:1033A00041E80002002AF3D100BF202084F8420047
:1033B0000020206300BF00BF21680C3151E8001FCE
:1033C00021F0100021680C3141E80002002AF3D1FD
:1033D00000BFE06BFEF72CF802206063A08DE28D49
:1033E000801A81B22046FFF7E6FE01E742E0A08D99
:1033F000E18D401A1FFA80F8E08DD0B3B8F1000FCC
:1034000037D000BF00BF21680C3151E8001F21F404
:10341000907021680C3141E80002002AF3D100BF0E
:1034200000BF00BF2168143151E8001F21F00100E6
:103430002168143141E80002002AF3D100BF2020A6
:1034400084F842000020206300BF00BF21680C31D7
:1034500051E8001F21F0100021680C3141E8000202
:10346000002AF3D100BF0220606341462046FFF7E7
:10347000A2FEBDE605F0800030B106F0800018B174
:10348000204601F06FFBB3E605F0400030B106F0D6
:10349000400018B1204601F08EF9A9E600BFA7E66A
:1034A0008146000810B504460CB9012010BDA06982
:1034B00000B100E000BF94F8410028B9002084F872
:1034C0004000204600F02AF8242084F841002068BB
:1034D000C06820F400502168C860204601F00CFA52
:1034E0002068006920F490402168086120684069E4
:1034F00020F02A00216848612068C06840F400502C
:103500002168C86000206064202084F8410084F8AD
:1035100042000020606300BFC8E7000010B586B01D
:103520000446142101A8FDF7F2F9E8492068884211
:1035300056D100BF00200090E548006840F400200C
:10354000E34908600846006800F40020009000BFCE
:1035500000BF00BF00200090DD481038006840F038
:103560000100DB49103908600846006800F00100DE
:10357000009000BF00BF03200190022002900020B5
:103580000390032004900820059001A9D148FEF77C
:10359000ADF9D148D14908604FF000604860402142
:1035A000CE4881600021C1604FF48061016100213B
:1035B00041618161C16101624162FEF7C3F808B1F6
:1035C000FDF702FD00BFC548A063846300BF02226F
:1035D00001213420FEF75AFC3420FEF743FC73E14E
:1035E000BF492068884259D100BF00200090B848E8
:1035F000001D006840F01000B549091D086008462C
:10360000006800F01000009000BF00BF00BF002065
:103610000090AF481038006840F00100AC49103904
:1036200008600846006800F00100009000BF00BF7D
:103630004FF4C0600190022002900020039003200C
:1036400004900720059001A9A248FEF74FF9A5486C
:10365000A54908604FF0006048604021A2488160A1
:103660000021C1604FF480610161002141618161ED
:10367000C16101624162FEF765F808B1FDF7A4FC83
:1036800000BF9948A063846300BF01221146252032
:10369000FEF7FCFB2520FEF7E5FB15E193492068CA
:1036A000884257D100BF002000908948006840F44C
:1036B0000030874908600846006800F40030009038
:1036C00000BF00BF00BF0020009081481038006894
:1036D00040F001007E49103908600846006800F09B
:1036E0000100009000BF00BF0C200190022002905A
:1036F00000200390032004900720059001A975483D
:10370000FEF7F4F874483030794908604FF00060F3
:1037100048604021764881600021C1604FF480619B
:103720000161002141618161C16101624162FEF775
:1037300009F808B1FDF748FC00BF6D48A063846339
:1037400000BF022201212620FEF7A0FB2620FEF763
:1037500089FBB9E067492068884258D100BF002042
:1037600000905B48006840F4802059490860084692
:10377000006800F48020009000BF00BF00BF002060
:10378000009053481038006840F00200504910394A
:1037900008600846006800F00200009000BF00BF0B
:1037A0004FF440600190022002900020039003201B
:1037B00004900720059001A94F48FEF797F8464866
:1037C00018384E4908604FF00060486040214B486F
:1037D00081600021C1604FF480610161002141617D
:1037E0008161C16101624162FDF7ACFF08B1FDF783
:1037F000EBFB00BF4148A063846300BF02220121AC
:103800002720FEF743FB2720FEF72CFB5CE03C491A
:103810002068884258D100BF002000902C48001D2D
:10382000006840F020002A49091D08600846006829
:1038300000F02000009000BF00BF00BF00200090FB
:1038400023481038006840F004002149103908600E
:103850000846006800F00400009000BF00BFC020D0
:103860000190022002900020039003200490082081
:10387000059001A92348FEF739F81A48183822495B
:1038800008604FF02060486040211F48816000219F
:10389000C1604FF480610161002141618161C161BA
:1038A00001624162FDF74EFF08B1FDF78DFB00BFDD
:1038B0001548A063846300BF022201214720FEF760
:1038C000E5FA4720FEF7CEFA06B010BD004C0040E6
:1038D000403802400000024070600240A80500200D
:1038E00000100140B8640240080600200044004077
:1038F000680600200048004000040240C80600207E
:1039000000140140000802402807002070B504465A
:103910000D46164694F8420020280BD105B10EB989
:10392000012070BD0020206332462946204601F068
:10393000F9F8F6E70220F4E710B5044606492068D6
:10394000884201D104F008FA04492068884201D174
:1039500003F076FE10BD000000100140004800405A
:103960002DE9F84F04460E46174699464FF0000AD7
:1039700094F84100202850D106B117B90120BDE8C4
:10398000F88F00206064212084F84100FEF7C0F821
:103990008246A784E784A068B0F5805F04D12069DF
:1039A00010B90025B04602E035464FF000081EE091
:1039B0005346002280212046CDF8009001F002F904
:1039C00020B1202084F841000320D8E745B9B8F899
:1039D0000000C0F308002168486008F1020803E015
:1039E0002878216848606D1CE08C401EE084E08CE3
:1039F0000028DDD15346002240212046CDF800901A
:103A000001F0E0F820B1202084F841000320B6E75F
:103A1000202084F841000020B1E70220AFE7000039
:103A2000F7B50446154694F84100202836D1019890
:103A300000B10DB90120FEBD01982062A584E58486
:103A400000206064212084F841001548A16BC86300
:103A50001448A16B08641448A16BC8640020A16BD2
:103A6000086501AE23681A1D31682B46A06BFDF76F
:103A7000DFFE6FF040002168086000BF00BF2168D2
:103A8000143151E8001F41F080002168143141E8F1
:103A90000002002AF3D100BF0020CCE70220CAE7D1
:103AA000E54600083D470008954600087047704706
:103AB00000BFFEE71FB50020009001900290039028
:103AC0001548164908604FF48030486000211348BB
:103AD00081600161017680F82010C1621049816225
:103AE0000021C1600121C161002180F83010012155
:103AF0004161FDF783FB08B1FDF766FA0A200090EB
:103B0000012001900320029069460448FDF7ACFAB9
:103B100008B1FDF759FA1FBD002001401402002032
:103B20000100000F08B500BF002000902648006883
:103B300040F48000244908600846006800F48000D2
:103B4000009000BF00BF00BF002000900846006842
:103B500040F4001008600846006800F4001000906F
:103B600000BF00BF002211460E20FEF78FF90E2085
:103B7000FEF778F9002211460F20FEF787F90F2093
:103B8000FEF770F9002211461120FEF77FF911208F
:103B9000FEF768F9002211463820FEF777F9382041
:103BA000FEF760F9002211464520FEF76FF9452027
:103BB000FEF758F9002211464620FEF767F9462025
:103BC000FEF750F908BD00003038024000B587B05C
:103BD000142102A8FCF79BFE00BF0020019074484E
:103BE000006840F01000724908600846006800F064
:103BF0001000019000BF00BF00BF002001900846E8
:103C0000006840F0040008600846006800F0040006
:103C1000019000BF00BF00BF00200190084600686F
:103C200040F0800008600846006800F080000190C5
:103C300000BF00BF00BF002001900846006840F0B0
:103C4000010008600846006800F00100019000BF14
:103C500000BF00BF002001900846006840F002004D
:103C600008600846006800F00200019000BF00BF35
:103C700000BF002001900846006840F0080008607E
:103C80000846006800F00800019000BF00BF002255
:103C900041F27F014748FDF735FF00224EF20271E5
:103CA0004548FDF72FFF002248F640114348FDF735
:103CB00029FF012241F610013F48FDF723FF0122B1
:103CC00015213F48FDF71EFF01224CF280013948C3
:103CD000FDF718FF002248F271213A48FDF712FF64
:103CE000012247F682013748FDF70CFF00224FF40E
:103CF00002713348FDF706FF4DF2FF0002900120EC
:103D0000039000200490059002A92A48FDF7EEFDDB
:103D10004FF612700290012003900020049005904D
:103D200002A92548FDF7E2FD41F2B0000290002013
:103D30000390049002A92148FDF7D8FD48F64010F1
:103D400002900120039000200490059002A91B48D6
:103D5000FDF7CCFD40F21D200290012003900020D1
:103D60000490059002A91648FDF7C0FD40F20C50E2
:103D7000029000200390049002A91248FDF7B6FDBE
:103D80004FF6F3200290012003900020049005904C
:103D900002A90C48FDF7AAFD4FF490700290002094
:103DA0000390049002A90648FDF7A0FD07B000BDEE
:103DB000303802400010024000080240000002407B
:103DC00000040240000C024010B50B480B4908608B
:103DD0000B484860002109488160C1604FF4804170
:103DE0000161002141618161C1610162FDF796FEBF
:103DF00008B1FDF7E9F810BD00540040BC020020F6
:103E0000A086010010B50E480E4908604FF482707C
:103E1000486000210B488160C160016141614FF43D
:103E2000802181610021C1610162416281620A21B8
:103E3000C162FEF70BFC08B1FDF7C6F810BD00002B
:103E4000003800401003002000B58FB0242106A8E0
:103E5000FCF75DFD00200490059000900190029019
:103E60000390224822490860002048600021204831
:103E700081604FF6FF71C160002101614161816184
:103E8000FFF746F808B1FDF79FF8032006900020E1
:103E9000079001200890002009900A900B900120C3
:103EA0000C9000200D900E9006A91148FEF7F5FE2B
:103EB00008B1FDF789F800200490059004A90C488A
:103EC000FEF7A8FD08B1FDF77FF800200090012063
:103ED0000190002002900390082269460448FEF7F2
:103EE000A8FF08B1FDF770F80FB000BD0000014059
:103EF000680300201CB50020009001900E480F4977
:103F000008605320486000210C48816040F2E7318E
:103F1000C16000218161FEF7D7FD08B1FDF754F8BB
:103F200000200090019069460448FEF773FD08B137
:103F3000FDF74AF81CBD000000100040B00300204F
:103F40001CB50020009001900E480F4908605320D6
:103F5000486000210C48816040F2E731C1600021D7
:103F60008161FEF7B1FD08B1FDF72EF80020009049
:103F7000019069460448FEF74DFD08B1FDF724F8AD
:103F80001CBD000000140040F803002010B50B48D1
:103F90000B4908604FF4E130486000210848816017
:103FA000C16001610C21416100218161C161FFF7A4
:103FB00079FA08B1FDF708F810BD0000004C004088
:103FC0004004002010B50B480B4908604FF4E13065
:103FD0004860002108488160C16001610C21416195
:103FE00000218161C161FFF75DFA08B1FCF7ECFFC8
:103FF00010BD0000001001408804002010B50B48DF
:104000000B4908604FF4E1304860002108488160A6
:10401000C16001610C21416100218161C161FFF733
:1040200041FA08B1FCF7D0FF10BD00000044004089
:10403000D004002010B50B480B4908604FF4E13064
:104040004860002108488160C16001610C21416124
:1040500000218161C161FFF725FA08B1FCF7B4FFC7
:1040600010BD0000004800401805002010B513489E
:10407000134908604FF4E130486000211048816026
:10408000C16001610C21416100218161C161FFF7C3
:1040900009FA08B1FCF798FF09480068C06840F0C9
:1040A000200007490968C86005480068C06840F0FA
:1040B000100003490968C86010BD000000140140E9
:1040C0006005002000BFFEE730B502464FF6FF70E6
:1040D00012B10446A14200D130BD11E012F8014BEB
:1040E000604000230AE000F0010424B140104AF2CD
:1040F0000104604000E040105C1CE3B2082BF2DBDE
:104100000C00A1F10105A9B2E8D100BFE4E700BFAE
:10411000FEE770477CB504460E461546334601223D
:1041200002212046009500F067F828B1606D40F04C
:104130002000606503207CBD164800681821B0FB94
:10414000F1F01549B0FBF1F04FF47A71484301905A
:104150006068B0F5827F0DD1334600228021204671
:10416000009500F049F898B1606D40F0200060655E
:104170000320E0E700BF019800B908E00198401E65
:10418000019020688068C0F3C0100028F3D100BF00
:104190000020D0E72800002040420F0070B5002426
:1041A000002522E06006040E012211021148FDF7ED
:1041B000A9FC0A2002F0A9FF4FF480510D48FDF739
:1041C0008FFC10B144F0010401E024F001040A2046
:1041D00002F09BFF00224FF480710648FDF792FC2D
:1041E0000A2002F092FF681CC5B2082DDADB2046D7
:1041F00070BD0000000002402DE9F84F04460D4656
:1042000090461E46DDF82890FDF782FCA0EB0900E1
:10421000371AFDF77DFC82462C480068C0F3CB308E
:104220007843009045E0701C002842D0FDF770FCF8
:10423000A0EB0A00B84200D2A7BB2068406820F07B
:10424000E000216848606068B0F5827F0DD1A06809
:10425000B0F5004F03D0A068B0F5806F05D120689D
:10426000006820F0400021680860A06AB0F5005F97
:104270000DD100BF2068006820F40050216808605C
:104280002068006840F400502168086000BF0120E9
:1042900084F8510000BF002084F8500000BF0320C4
:1042A000BDE8F88FFFE7009800B900270098401E8E
:1042B0000090206880682840A84201D1012000E0D9
:1042C00000204045AFD10020EAE700002800002090
:1042D00070B50446002526E00A2002F016FF04F01F
:1042E000800028B10122D1021048FDF70BFC05E047
:1042F00000224FF400610D48FDF704FC0122110279
:104300000A48FDF7FFFB0A2002F0FFFE6006040EDC
:1043100000224FF480710548FDF7F4FB0A2002F0FB
:10432000F4FE681CC5B2082DD6DB70BD000002404B
:10433000704710B5FDF71EFD10BD000000B593B02D
:10434000302107A8FCF7E3FA142102A8FCF7DFFAF2
:1043500000BF002001902448006840F080502249AE
:1043600008600846006800F08050019000BF00BF60
:1043700000BF002001901D48006840F480401B49A8
:1043800008600846006800F48040019000BF00BF4C
:10439000012007900004089002200D9041050E9125
:1043A00004210F91A8211091022111910421129151
:1043B00007A8FDF7FDFE08B1FCF706FE0F200290EE
:1043C00002200390002004904FF4A05005904FF479
:1043D00080500690052102A8FDF7AAFD08B1FCF760
:1043E000F3FD13B000BD00004038024000700040F3
:1043F0000348006840F470000149086070470000FD
:1044000088ED00E010B50248FEF7FAFD10BD00008F
:10441000B003002010B50248FEF7F2FD10BD000009
:10442000F803002010B502682D4B98420ED0B0F171
:10443000804F0BD02B4B984208D02B4B984205D085
:104440002A4B984202D02A4B984203D122F07002A4
:104450004B681A43224B984220D0B0F1804F1DD0B8
:10446000204B98421AD0204B984217D01F4B9842AD
:1044700014D01F4B984211D01E4B98420ED01E4BA9
:1044800098420BD01D4B984208D01D4B984205D046
:104490001C4B984202D01C4B984203D122F440722C
:1044A000CB681A4322F080034C6943EA040202609D
:1044B0008B68C3620B688362094B984202D00C4B35
:1044C000984201D10B69036301234361036903F03F
:1044D00001031BB1036923F00103036110BD000058
:1044E000000001400004004000080040000C0040B3
:1044F00000040140004001400044014000480140E8
:1045000000180040001C00400020004030B501F0C1
:104510001F05012404FA05F3046A9C430462046A3B
:1045200001F01F0502FA05F52C43046230BD0000BE
:1045300070B50C461546026A066A26F00106066248
:104540008169184EB04214D0B0F1804F11D0164E90
:10455000B0420ED0154EB0420BD0154EB04208D02E
:10456000144EB04205D0144EB04202D0134EB042A9
:1045700001D1012600E000261EB121F003012943EC
:1045800001E041F0010121F0F001F02606EA0316F6
:10459000314322F00A0204F00A06324381610262CA
:1045A00070BD000000000140000400400008004011
:1045B000000C004000040140004001400018004091
:1045C00070B50C461546026A066A26F010060662A9
:1045D000816921F4407141EA052121F470414FF4D1
:1045E000704606EA0336314322F0A002A02606EA0E
:1045F000041632438161026270BD70B50C461546E7
:10460000026A066A26F480760662C16921F0030117
:10461000294321F0F001F02606EA0316314322F483
:1046200020624FF4206606EA04263243C16102622A
:1046300070BD70B50C461546026A066A26F48056AF
:104640000662C16921F4407141EA052121F47041FB
:104650004FF4704606EA0336314322F420424FF409
:10466000204606EA04363243C161026270BD000092
:1046700010B50248FEF7A2FD10BD00004004002066
:1046800070B50546AC6B0020E085E0842046FEF75F
:1046900093FD70BD70B506460025B46B2068406977
:1046A000C0F3C01594F84100212805D125B10020A0
:1046B000E084204600F08FF820684069C0F3801540
:1046C00094F84200222805D125B10020E08520463B
:1046D00000F03BF8606C40F0100060642046FEF78C
:1046E0006BFD70BD70B50546AC6B2868006800F4C2
:1046F0008070F8B90020E08400BF00BF2168143149
:1047000051E8001F21F080002168143141E80002C7
:10471000002AF3D100BF00BF00BF21680C3151E86F
:10472000001F41F0400021680C3141E80002002ADE
:10473000F3D102E02046FFF7B9F970BD70B5044629
:10474000A56B2846FFF7B3F970BD00BF00BF026834
:104750000C3252E8002F22F4907102680C3242E8C9
:104760000013002BF3D100BF00BF00BF026814325A
:1047700052E8002F22F001010268143242E80013CF
:10478000002BF3D100BF016B01290ED100BF00BF88
:1047900002680C3252E8002F22F0100102680C323D
:1047A00042E80013002BF3D100BF202180F8421013
:1047B00000210163704710B504462068C06820F0EE
:1047C00040002168C860202084F841002046FFF79F
:1047D0006DF9002010BD00BF00BF02680C3252E826
:1047E000002F22F0C00102680C3242E80013002BB7
:1047F000F3D100BF202180F841107047F8B504467E
:1048000094F84200222875D1A068B0F5805F0CD1E1
:10481000206950B90025A66A20684068C0F30800E6
:104820003080A06A801CA06215E0A56A0026A068FE
:10483000B0F5805F03D0A06828B9206918B9206856
:104840004068287004E02068406800F07F0028700D
:10485000A06A401CA062E08D401E80B2E085002866
:1048600046D12068C06820F020002168C860206818
:10487000C06820F480702168C8602068406920F01A
:10488000010021684861202084F842000020606314
:10489000206B012826D10020206300BF00BF2168C3
:1048A0000C3151E8001F21F0100021680C3141E863
:1048B0000002002AF3D100BF2068006800F0100059
:1048C00010280AD100BF00200090206800680090E6
:1048D00020684068009000BF00BFA18D2046FEF711
:1048E0006AFC02E02046FFF727F80020F8BD01E04F
:1048F0000020FBE70220F9E72DE9F84F0446206885
:10490000006920F44050E16808432168086121698A
:10491000A068084361690843E16908430090206882
:10492000C06849F20C618843009908432168C86057
:104930002068406920F44070A169084321684861FB
:1049400076492068884203D075492068884203D19F
:10495000FDF7C6FB814602E0FDF7B2FB8146E06948
:10496000B0F5004F6CD102206168A0FB01500346F6
:104970001920A9FB007001462A463846FBF7A4FC23
:104980006421B0FBF1F04FEA001A02206168A0FB3D
:1049900001510B461920A9FB00712A463846FBF746
:1049A00093FC834602206168A0FB01500346192056
:1049B000A9FB00712A463846FBF786FC6421B0FB50
:1049C000F1F000EBC00101EB0010ABEB80003221F5
:1049D00001EBC0006421B0FBF1F000F0F8000AEB3D
:1049E000400A02206168A0FB015003461920A9FB80
:1049F000007001462A463846FBF766FC83460220D3
:104A00006168A0FB015003461920A9FB00712A46EA
:104A10003846FBF759FC6421B0FBF1F000EBC00114
:104A200001EB0010ABEB8000322101EBC0006421F0
:104A3000B0FBF1F000F007005044216888606AE0A4
:104A400004206168A0FB015003461920A9FB0070F7
:104A500001462A463846FBF737FC82460420616847
:104A6000A0FB015003461920A9FB007001462A460D
:104A70003846FBF729FC6421B0FBF1F000EBC001E4
:104A800001EB0010AAEB8000322101EB0010642141
:104A9000B0FBF1F000F0F00A04206168A0FB0170A7
:104AA00003461920A9FB00513A462846FBF70CFCA7
:104AB0006421B0FBF1F00AEB001A04206168A0FB4E
:104AC00001510B461920A9FB00712A463846FBF715
:104AD000FBFB834604206168A0FB015003461920BC
:104AE000A9FB007001462A463846FBF7EDFB64211E
:104AF000B0FBF1F000EBC00101EB0010ABEB80006C
:104B0000322101EB00106421B0FBF1F000F00F0046
:104B1000504421688860BDE8F88F00000010014013
:104B20000014014010B5034699629A85DA85002089
:104B30005864222083F84200186928B11868C068B8
:104B400040F480701C68E0601868406940F0010023
:104B50001C6860611868C06840F020001C68E06054
:104B6000002010BD014691F84100212828D1886815
:104B7000B0F5805F0BD1086948B90A6A1088C0F3A4
:104B800008000B685860086A801C086205E00B6A20
:104B9000581C086218780B685860C88C401E80B298
:104BA000C88458B90868C06820F080000B68D860D5
:104BB0000868C06840F040000B68D860002070476B
:104BC0000220FCE72DE9F84304460D4617469846B7
:104BD000089E31E0701C70B3FCF79AFFA0EB080050
:104BE000B04200D816B90320BDE8F8832068C06839
:104BF00000F00400F8B1802D1ED0402D1CD020689C
:104C00000068C0F3C000B0B100BF00200090206871
:104C10000068009020684068009000BF00BF2046F8
:104C2000FFF793FD0820606400BF002084F8400077
:104C300000BF0120D8E7FFE7206800682840A842AD
:104C400001D1012000E00020B842C3D00020CBE712
:104C500010B50248FEF7B2FA10BD0000880400202B
:104C600010B50248FEF7AAFA10BD0000D0040020DB
:104C700010B50248FEF7A2FA10BD0000180500208A
:104C800010B50248FEF79AFA10BD0000600500203A
:104C900000BFFEE70246024B23F8121070470000E7
:104CA000CE00002070B50A46B2F57F4F19D1A0F1B1
:104CB0001001CC1701EB5474E410174D2C5D0B461A
:104CC000DD1703EB5575ED10A3EBC5060125B540C7
:104CD0002C43E5B2CC1701EB5474E4100E4E35555D
:104CE00018E0BAB9A0F11001CC1701EB5474E4102C
:104CF000094D2C5D0B46DD1703EB5575ED10A3EB4D
:104D0000C5060125B540AC43CD1701EB5575ED1037
:104D1000014E745570BD0000C008002010B501227E
:104D200091030448FCF7EEFE012251030148FCF711
:104D3000E9FE10BD000C024070B5002400224FF4C3
:104D400080411A48FCF7DEFE012002F0E5F901225D
:104D500091031648FCF7D6FE012002F0DDF9802110
:104D60001348FCF7BDFE012801D144F001040025E1
:104D700018E0640000224FF400510C48FCF7C2FE1A
:104D8000012002F0C9F9012251030848FCF7BAFEDC
:104D900080210748FCF7A4FE012801D144F001045A
:104DA000681CC5B20F2DE4DBA0B270BD000C024040
:104DB0000000024002480068C0F302207047000073
:104DC0000CED00E010B5002804DB0A07130E054ABD
:104DD000135406E00A07140E034A00F00F031B1FCA
:104DE000D45410BD00E400E018ED00E030380A288B
:104DF00001D20120704700207047000006200149C1
:104E0000087070479C08002000BF704710B511481B
:104E1000FCF768FA0F48FCF7EDF90F490F4A1268E2
:104E200041F82200084690ED000AB8EE400ADFED96
:104E30000C0A60EE200A9FED0B1A80EE810ADFED6E
:104E40000A0A80EE201ABCEEC10A10EE100A0749C9
:104E5000088310BD14020020FC1A0020C4010020A9
:104E600000404E4500F07F459EEFA73DD60800204C
:104E70007047000010B5C348007830B1012862D0F7
:104E800002287DD003285DD11CE100F0F5F9BE4970
:104E9000BC4A127841F822000846BA49097850F80D
:104EA000210000EE100AB8EEC00AF0EE040A20EE6F
:104EB000200ADFEDB60A80EE201A9FEDB50A21EE3A
:104EC000000ABDEEC00A10EE100AAE49097801EBE7
:104ED0008101B04A02EBC101AF4A126841F82200D9
:104EE000AD480068401CAC490860084600680928C5
:104EF00001DD00200860002010E0A249097801EBE4
:104F00008101A44A02EBC10151F82010CA17A34C39
:104F100018CCC9186241A14B06C3401C0A28ECDB1F
:104F20000A2200239D4903C9FBF745FA9C490882E0
:104F300000209A4A10605060012092490870912028
:104F400000F0BCF91CE100F097F98F498D4A127806
:104F500041F8220008468B49097850F8210000EEFC
:104F6000100AB8EEC00AF0EE040A20EE200A9FED07
:104F7000871AC0EE010A9FED860A20EE800A00E043
:104F800042E0BDEEC00A10EE100A7E49097801EB3E
:104F90008101804A02EBC101824A126841F8220075
:104FA00080480068401C7F4908600846006809285E
:104FB00001DD00200860002011E07249097801EB52
:104FC0008101744A02EBC10151F82010CA17734BDA
:104FD000D3E9004309195A41704B06C3401C0A2803
:104FE000EBDB0A2200236D4903C9FBF7E4F96C49A6
:104FF00048820021694A11605160022061490870AD
:10500000A12000F05BF9BBE000F036F95E495D4A93
:10501000127841F8220008465A49097850F82100D0
:1050200000EE100AB8EEC00AF0EE040A20EE200AE4
:10503000DFED560A80EE201A9FED550A21EE000A98
:10504000BDEEC00A10EE100A4E49097801EB81014D
:10505000504A02EBC101544A126841F822005248FA
:105060000068401C5049086008460068092801DDB6
:1050700000200860002010E04249097801EB81011E
:10508000444A02EBC10151F82010CA17434C18CC16
:10509000C9186241414B06C3401C0A28ECDB0A22B6
:1050A00000233E4903C9FBF786F93D498882002069
:1050B0003A4A10605060032032490870B12000F075
:1050C000FDF85DE000F0D8F82F492E4A127841F83B
:1050D000220008462B49097850F8210000EE100AFA
:1050E000B8EEC00AF0EE040A20EE200A9FED271A5F
:1050F000C0EE010A9FED260A20EE800ABDEEC00A2E
:1051000010EE100A1F49097801EB8101214A02EBD8
:10511000C101264A126841F8220024480068401C58
:105120002249086008460068092801DD002008605F
:10513000002010E01349097801EB8101154A02EBC8
:10514000C10151F82010CA17144C18CCC91862417B
:10515000124B06C3401C0A28ECDB0A2200230F492D
:1051600003C9FBF728F90E49C88200210B4A1160D8
:105170005160002003490870812000F09FF800BFB3
:1051800000BF10BD58000020880700200000004B21
:1051900000401C46980700204800002060000020C6
:1051A000D60800204C0000205000002054000020B1
:1051B0001FB581200390C020029040200190002064
:1051C0000090002202211748FCF79CFC062000F00A
:1051D00089F80A2001F094FF012202211148FCF70E
:1051E00091FC03AA0121002000F0B6F802AA0121D7
:1051F000084600F0B1F801AA0121022000F0ACF845
:105200006A460121032000F0A7F800220221054888
:10521000FCF778FC0A2001F073FF082000F062F828
:105220001FBD0000000C024070B5002400220121C7
:105230001048FCF767FC002518E0012211460D48D4
:10524000FCF760FC6006040E08210A48FCF748FCE5
:105250000443022001F060FF002201210548FCF711
:1052600051FC022001F058FF681CC5B2082DE4DB98
:10527000204670BD000C024010B5002202210E48ED
:10528000FCF740FC102000F02DF8FFF7CDFF04469E
:10529000FFF7CAFF40EA0424FFF7C6FF40EA0424F0
:1052A00004F4000008B144F07F44012202210248C6
:1052B000FCF728FC204610BD000C024001B56A46F0
:1052C0000121002000F048F8082000F00BF800BF92
:1052D00004210348FCF704FC0028F9D108BD0000B4
:1052E000000C024070B50446002201211948FCF769
:1052F00009FC002529E004F0800028B101221021DA
:105300001448FCF7FFFB04E0002210211148FCF7D1
:10531000F9FB6006040E012001F0FEFE0122114699
:105320000C48FCF7EFFB022001F0F6FE0022012101
:105330000848FCF7E7FB012001F0EEFE08210548D4
:10534000FCF7CEFB0443681CC5B2082DD3DB204616
:1053500070BD0000000C02402DE9F04106460C46ED
:105360001546002202210F48FCF7CCFB0C2101EA74
:105370008601621E02F00302114341F04000FFF774
:10538000B1FF002704E015F8010BFFF7ABFF7F1C0E
:10539000A742F8DB012202210248FCF7B3FBBDE87B
:1053A000F0810000000C024010B52DED0A8BCC48B6
:1053B0000068082835D2DFE800F004356697C8FC9D
:1053C000FAF90120FBF758FCB0EE40CAF0EE60CAD3
:1053D0009FEDC40B53EC102B51EC1C0B04F030FC74
:1053E00041EC1B0B9FEDC10B53EC102B04F08CFA1E
:1053F00041EC1A0B9FEDBF0B53EC102B04F01EFD7C
:1054000041EC190B9FEDBD0B53EC102B04F07CFA13
:1054100041EC180B04F0D0FBBA4908800120B049D8
:10542000086059E10220FBF727FCB0EE40CAF0EE1D
:1054300060CA9FEDAC0B53EC102B51EC1C0B04F02D
:10544000FFFB41EC1B0B9FEDA90B53EC102B04F061
:105450005BFA41EC1A0B9FEDA70B53EC102B04F0F9
:10546000EDFC41EC190B9FEDA50B53EC102B04F058
:105470004BFA41EC180B04F09FFBA2494880022034
:105480009749086028E10320FBF7F6FBB0EE40CA1D
:10549000F0EE60CA9FED930B53EC102B51EC1C0BFC
:1054A00004F0CEFB41EC1B0B9FED900B53EC102B4B
:1054B00004F02AFA41EC1A0B9FED8E0B53EC102BE3
:1054C00004F0BCFC41EC190B9FED8C0B53EC102B42
:1054D00004F01AFA41EC180B04F06EFB894988803D
:1054E00003207F490860F7E00420FBF7C5FBB0EE1E
:1054F00040CAF0EE60CA9FED7B0B53EC102B51ECD1
:105500001C0B04F09DFB41EC1B0B9FED780B53EC47
:10551000102B04F0F9F941EC1A0B9FED760B53ECCC
:10552000102B04F08BFC41EC190B9FED740B53EC2A
:10553000102B04F0E9F941EC180B04F03DFB714924
:10554000C880042066490860C6E00520FBF794FB8C
:10555000B0EE40CAF0EE60CA9FED620B53EC102B28
:1055600051EC1C0B04F06CFB41EC1B0B9FED5F0B33
:1055700053EC102B04F0C8F941EC1A0B9FED5D0BB6
:1055800053EC102B04F05AFC41EC190B9FED5B0B14
:1055900053EC102B04F0B8F941EC180B04F00CFBA1
:1055A0005849088105204E49086095E063E031E0E4
:1055B000FFE70620FBF760FBB0EE40CAF0EE60CAE2
:1055C0009FED480B53EC102B51EC1C0B04F038FBF7
:1055D00041EC1B0B9FED450B53EC102B04F094F9A1
:1055E00041EC1A0B9FED430B53EC102B04F026FCFF
:1055F00041EC190B9FED410B53EC102B04F084F997
:1056000041EC180B04F0D8FA3E4948810620344991
:10561000086061E00720FBF72FFBB0EE40CAF0EE18
:1056200060CA9FED300B53EC102B51EC1C0B04F0B7
:1056300007FB41EC190B9FED2D0B53EC102B04F0E5
:1056400063F941EC1B0B9FED2B0B53EC102B04F07B
:10565000F5FB41EC180B9FED290B53EC102B04F0DC
:1056600053F941EC1A0B04F0A7FA26498881072068
:105670001B49086030E00020FBF7FEFAB0EE40CA9C
:10568000F0EE60CA9FED170B53EC102B51EC1C0B86
:1056900004F0D6FA41EC1B0B9FED140B53EC102BCE
:1056A00004F032F941EC1A0B9FED120B53EC102B66
:1056B00004F0C4FB41EC180B9FED100B53EC102BC6
:1056C00004F022F941EC190B04F076FA0D49C88177
:1056D00000200349086000BF00BFBDEC0A8B10BD6D
:1056E0004400002000000000000024403D0AD7A331
:1056F000703DEA3F0000000000C06240AE47E17A22
:1057000014AEEF3FD608002010B500221021124839
:10571000FCF7F8F9012208210F48FCF7F3F90621FC
:105720000020FBF773FB08210120FBF76FFB002132
:105730000220FBF76BFBA1210320FBF767FB002195
:105740000420FBF763FBF02000F036F80022102164
:105750000148FCF7D7F910BD0004024070B50024E1
:10576000002201211248FCF7CDF900251CE001229E
:1057700011460F48FCF7C6F9012001F0CDFC600688
:10578000040E4FF480710B48FCF7AAF90443012082
:1057900001F0C2FC002201210548FCF7B3F9022008
:1057A00001F0BAFC681CC5B2082DE0DB204670BDD4
:1057B000001002400004024070B50446002201219E
:1057C0001A48FCF79FF900252BE0012211461748E3
:1057D000FCF798F9012001F09FFC04F0800028B14B
:1057E000012251021248FCF78DF905E000224FF426
:1057F00000710F48FCF786F96006040E012001F0E5
:105800008BFC002201210948FCF77CF9022001F001
:1058100083FC4FF480710648FCF762F90443681C6E
:10582000C5B2082DD1DB204670BD0000001002403B
:105830000004024010B52DED028BB0EE408A00242A
:105840009FED0C0A28EE000AB0EE408A9FED0A0A8E
:1058500028EE000ADFED090A80EE201ABCEEC10A2C
:1058600010EE100A84B20221204600F059F8BDEC77
:10587000028B10BD0000C8420000804500404E452C
:1058800010B52DED028BB0EE408A00249FED0C0A7E
:1058900028EE000AB0EE408A9FED0A0A28EE000AC0
:1058A000DFED090A80EE201ABCEEC10A10EE100AE4
:1058B00084B20321204600F033F8BDEC028B10BD0A
:1058C0000000C8420000804500404E4510B52DED57
:1058D000028BB0EE408A00249FED0D0A28EE000AEC
:1058E000B0EE408A9FED0B0A28EE000ADFED0A0AAF
:1058F00080EE201ABCEEC10A10EE100A84B20748EE
:1059000004600121204600F00BF8BDEC028B10BDB5
:105910000000C8420000804500404E45680000205D
:105920002DE9F04107460C464FF6FF7000EA870567
:10593000C5F30D05012C15D1012280214A48FCF741
:10594000E1F8012240214848FCF7DCF80A2001F088
:10595000DCFB002280214448FCF7D4F80A2001F047
:10596000D4FB2FE0022C15D1012211033F48FCF794
:10597000C9F8012291023D48FCF7C4F80A2001F061
:10598000C4FB0022E1023948FCF7BCF80A2001F010
:10599000BCFB17E0032C15D10122D1023348FCF7E0
:1059A000B1F8012291023148FCF7ACF80A2001F06D
:1059B000ACFB00224FF400612C48FCF7A3F80A204E
:1059C00001F0A3FB00263BE0012240212648FCF722
:1059D00099F8012291022548FCF794F805F400405B
:1059E000B0F5004F0AD1012220211F48FCF78AF8A8
:1059F0000122D1031E48FCF785F80AE0002220218D
:105A00001948FCF77FF800224FF400411848FCF7D2
:105A100079F80A2001F079FB002240211248FCF7B6
:105A200071F800224FF480611048FCF76BF80A20EF
:105A300001F06BFB4FF6FF7000EA4505701CC6B223
:105A4000102EC1DB012280210748FCF75BF8012200
:105A500011030648FCF756F80122D1020348FCF76F
:105A600051F8BDE8F0810000000C0240000802403F
:105A70000000024070B50546002600243D2000F0DD
:105A80003BFF284600F052FF012211030B48FCF7B0
:105A900039F80FE00520FBF715FF00F023F9044665
:105AA000102C00D007E03046711CCEB2C82801DDB2
:105AB000FA2070BDEEE700BF2046FAE7000402407E
:105AC00070B50446062000F017FF204600F02EFFB8
:105AD00000F0A0FB0546012211030248FCF712F872
:105AE000284670BD0004024010B5192000F004FFE4
:105AF000022001F011FB00F08DFB044600F08AFB50
:105B000004EB002084B2012211030248FBF7FAFFE4
:105B1000204610BD0004024010B5262000F0ECFE27
:105B200000F078FB0446012211030248FBF7EAFF6C
:105B3000204610BD0004024070B50446282000F045
:105B4000DBFE002505E000F065FB04F8010B681C96
:105B5000C5B2082DF7DB012211030248FBF7D2FF83
:105B600070BD00000004024010B5012000F0C4FE2A
:105B700000F050FB0446012211030248FBF7C2FF6C
:105B8000204610BD0004024070B5002500242720E7
:105B900000F0B2FE012211030B48FBF7B3FF0FE048
:105BA0000A20FBF78FFE00F09DF80446102C00D071
:105BB00007E02846691CCDB2C82801DDFA2070BD77
:105BC000EEE700BF2046FAE70004024010B50520CA
:105BD00000F092FE012211030148FBF793FF10BD74
:105BE0000004024070B50446232000F085FE002525
:105BF00005E014F8010B00F099FE681CC5B2042DF5
:105C0000F7DB012211030248FBF77CFF70BD0000A7
:105C10000004024070B50446222000F06DFE00250D
:105C200005E014F8010B00F081FE681CC5B2042DDC
:105C3000F7DB012211030248FBF764FF70BD00008F
:105C40000004024070B50446242000F055FE0025F3
:105C500005E014F8010B00F069FE681CC5B2042DC4
:105C6000F7DB012211030248FBF74CFF70BD000077
:105C70000004024070B505460026412000F03CFEBD
:105C8000284600F053FE012211030C48FBF73AFFAF
:105C90000FE01420FBF716FE00F024F80446102C49
:105CA00000D007E03046711CCEB2C82801DDFA20D2
:105CB00070BDEEE700BF2046FAE700000004024096
:105CC00010B5044604B910BD214602A0FAF798FBAE
:105CD00000BFF8E74572726F723A20253032580DD6
:105CE0000A00000010B52C2000F006FE00F092FA29
:105CF0000446012211030248FBF704FF204610BDB1
:105D0000000402402DE9F04107460C4615460CB947
:105D1000BDE8F0813C2000F0EFFD384600F006FEC3
:105D2000E0B200F003FE201200F000FE012001F0BE
:105D3000F3F9002605E000F06DFA28706D1C701C68
:105D400086B2A642F7DB012211030248FBF7DAFE16
:105D500000BFDDE70004024070B505463B2000F0BF
:105D6000CBFD284600F0E2FD00F054FA044600F0B6
:105D700051FA04EB002084B2012211030248FBF720
:105D8000C1FE204670BD00000004024070B504460C
:105D9000302000F0B1FD204600F0C8FD022001F0E7
:105DA000BBF900F037FA0546012211030248FBF760
:105DB000A9FE284670BD00000004024000B587B06F
:105DC00000BF00BF002001903348006840F004008D
:105DD000314908600846006800F00400019000BFE7
:105DE00000BF00BF00BF00BF002001900846006850
:105DF00040F0080008600846006800F008000190C4
:105E000000BF00BF00BF00BF00BF002001900846D8
:105E1000006840F0080008600846006800F00800CC
:105E2000019000BF00BF00BF8814029001200590C0
:105E3000039002A91948FBF759FD00224FF4805145
:105E40001648FBF75FFE4FF480700290002003902D
:105E5000012004900220059002A91148FBF746FD9D
:105E60004FF4007002900120039002200590012061
:105E7000049002A90A48FBF739FD012251020848A3
:105E8000FBF740FE012211030648FBF73BFE1420FE
:105E9000FBF718FD07B000BD303802400004024097
:105EA000000C02400010024070B5FFF787FFFDF7BD
:105EB000A9FF2B482B49C1F858022B48C1F85C02B6
:105EC0002A48C1F86002022088706520FFF7F8FDBB
:105ED00004469A2C04D02348D0F85812204688470C
:105EE000FFF774FE6420FBF7EDFCFFF74DFE05465F
:105EF0001C48D0F858122846884700F05FFC00BFC5
:105F0000FFF70AFE174948700A465078D2F85C122B
:105F1000884717480068401C154908600846006813
:105F2000322802DD40200F4948700E484078012891
:105F3000E6D0FFF719FE0B490870084601780DA05E
:105F4000FAF75EFA0120FFF795FE04460548D0F8FF
:105F50005812204688474FF47A70FBF7B3FC70BDA7
:105F6000C15C0008581200205D610008356200081D
:105F7000980100204348333935564552203A2025B0
:105F800032780D0A0000000010B500BF00F0D4FC0C
:105F9000124880780228F9D00220114908700020A8
:105FA000487008460F49096841630F4909688163D1
:105FB0000E490968C16341F6907009494881022081
:105FC00088700B48C8601621054801610949816144
:105FD0004FF48061C16100F0C1FC10BD5812002077
:105FE000BC1800209C010020A0010020A40100207A
:105FF000A8010020BC14002010B5FFF775FD044671
:1060000004F0010010B12248FFF796FD04F00400EF
:1060100020B1FFF781FD1E49C91E487004F0080039
:1060200020B101201A49C91E887010BD04F010006B
:1060300010B1002000F0FEFA04F0200010B10120A1
:1060400000F0F8FA04F0400010B1022000F0F2FA7B
:1060500004F0800010B1032000F0ECFA04F480702A
:1060600010B1042000F0E6FA04F4007010B105202D
:1060700000F0E0FA04F4806010B1062000F0DAFAD3
:1060800004F4006010B1072000F0D4FA00BFCCE7A0
:106090005B12002010B50446582000F02DFC20466D
:1060A00000F044FC10BD10B50446562000F024FC5E
:1060B000E0B200F03BFCC4F3072000F037FCC4F36F
:1060C000074000F033FC200E00F030FC10BD10B58E
:1060D0000446572000F010FCE0B200F027FCC4F3A7
:1060E000072000F023FCC4F3074000F01FFC200E43
:1060F00000F01CFC10BD10B5C820FFF7CBFF43F625
:106100009820FFF7D0FF43F69820FFF7E0FF10BD7F
:1061100070B5054600260024352000F0EDFB28462A
:1061200000F004FC012211030B48FBF7EBFC0FE02D
:106130000520FBF7C7FBFFF7D5FD0446102C00D068
:1061400007E03046711CCEB2C82801DDFA2070BDD0
:10615000EEE700BF2046FAE70004024010B504460F
:10616000042C12D004DC012C07D0022C19D108E039
:10617000082C0ED0102C14D10FE00FA0FAF740F924
:1061800013E011A0FAF73CF90FE013A0FAF738F981
:106190000BE015A0FAF734F907E017A0FAF730F989
:1061A00003E019A0FAF72CF900BF00BF4FF47A7092
:1061B000FBF788FB10BD0000504859204449534369
:1061C0004F4E4E0D0A0000005048592031304D5FAF
:1061D000464C4C0D0A0000005048592031304D5FAC
:1061E00048414C460D0A0000504859203130304D8E
:1061F0005F464C4C0D0A0000504859203130304D5C
:106200005F48414C460D0A00504859204155544FB3
:106210000D0A000010B5FF2000F003F804462046E8
:1062200010BD70B50446204602F076FB05462846B0
:1062300070BD000070B500242BE19848407801281B
:106240002FD19648807838B194488078012803D0BF
:1062500092488078022824D104EBC4018F4818307A
:1062600010F8310002281BD104EBC4028B4918310D
:1062700001EBC2014878FFF7FDFB0020FFF7FAFCB5
:1062800005468648D0F8581228468847012104EB75
:10629000C4028248183000F8321002207F4988700A
:1062A000F5E07E4840780128FAD004EBC4017B4831
:1062B000183010F831000128F2D17848807802288F
:1062C00014D1FFF783FC6420FBF7FCFAFFF75CFCBA
:1062D0006420FBF7F7FA00F071FA0120FFF7CAFC1F
:1062E00005466E48D0F858122846884700BF4FF43C
:1062F00080716B48FBF7F4FB08B9FFF77DFE674838
:1063000080780228F3D004EBC4016448183000EB15
:10631000C100807830B1012830D0022865D0032830
:106320007DD18FE004EBC4025C48183000EBC20062
:10633000C11C204600F0E8F80221204600F01EF9BA
:1063400004EBC4025548183000EBC2000189204616
:1063500000F0FCF804EBC4025048183000EBC20017
:106360004189204600F040F92046FFF7D1FE05465E
:106370004A48D0F858122846884780E0FFF7BBFE0D
:1063800004EBC4024548183000EBC200C11C204693
:1063900000F0BAF80321204600F0F0F804EBC40244
:1063A0003E48183000EBC2000189204600F0CEF8CC
:1063B00004EBC4023948183000EBC2004189204682
:1063C00000F012F92046FFF7A3FE05463348D0F847
:1063D000581228468847204600F042FA05462F48C2
:1063E000D0F858122846884749E004EBC4022B48ED
:1063F000183000EBC200C11C204600F085F80321D4
:10640000204600F0BBF804EBC4022448183000EB2F
:10641000C2004189204600F0E7F8204600E01FE076
:10642000FFF776FE05461D48D0F8581228468847E3
:10643000204600F03BFA05461848D0F85812284686
:1064400088471CE00121204600F098F82046FFF71D
:106450005FFE05461148D0F85812284688470EE0DE
:106460000321204600F08AF804EBC4020B481830E0
:1064700000EBC2004189204600F0B6F800BF00BF23
:10648000022104EBC4020548183000F83210601CE9
:10649000C4B2072C7FF7D1AE70BD000058120020A7
:1064A000000C02402DE9F04107460D461446392004
:1064B00000F022FA384600F039FAE0B200F036FA7D
:1064C000201200F033FA002605E015F8010B00F069
:1064D0002DFA701C86B2A642F7DB01221103024896
:1064E000FBF710FBBDE8F0810004024070B50546E3
:1064F0000C46592000F000FA284600F017FA204612
:1065000000F014FA70BD000070B505460C4631204D
:1065100000F0F2F9284600F009FA14F8010B00F037
:1065200005FA14F8010B00F001FA14F8010B00F061
:10653000FDF914F8010B00F0F9F9012211030248EA
:10654000FBF7E0FA70BD00000004024070B505469C
:106550000C46322000F0D0F9284600F0E7F9E0B20E
:1065600000F0E4F9201200F0E1F9012211030248E1
:10657000FBF7C8FA70BD00000004024070B5054684
:106580000C46342000F0B8F9284600F0CFF9204638
:1065900000F0CCF9012211030148FBF7B3FA70BDFA
:1065A0000004024070B506460C461546522000F025
:1065B000A3F9304600F0BAF9204600F0B7F92846B2
:1065C00000F0B4F970BD70B506460C461546532070
:1065D00000F092F9304600F0A9F9204600F0A6F943
:1065E000284600F0A3F970BD70B505460C4633206F
:1065F00000F082F9284600F099F9E0B200F096F92F
:10660000201200F093F9012211030248FBF77AFAF5
:1066100070BD00000004024070B505460C465120D4
:1066200000F06AF9284600F081F9204600F07EF972
:1066300070BD00002DE9F041044600262046FFF71A
:10664000A5FB054605F0040088B32046FFF784FB50
:1066500004EBC402584901EBC201C86104EBC40158
:10666000554800EBC100808B86B204EBC401524850
:1066700000EBC100314682692046FFF743FB002151
:1066800004EBC4024C4800EBC2008069815501F064
:1066900027FB04EBC401484800EBC100007D40F03B
:1066A000040104EBC402444800EBC200017505F08C
:1066B000080078B104EBC4013F4800EBC1008078CA
:1066C000012807D101212046FFF710FF3C21204679
:1066D000FFF7A2FF05F01000C8B304EBC40236496F
:1066E00001EBC2014878FFF713FD0746324818381E
:1066F000D0F858123846884704EBC4012E4800EB06
:10670000C1008078012802D0022821D10FE004EBDB
:10671000C402294901EBC201487800F0A1F80746FC
:1067200025481838D0F858123846884711E004EB4D
:10673000C402214901EBC201487800F0B7F80746CE
:106740001D481838D0F858123846884701E004E050
:1067500000BF00BFC820FBF7B5F805F0400040B30C
:1067600004EBC401144800EBC1008078012820D15B
:10677000C820FBF7A7F804EBC4020F4901EBC201E4
:106780004878FFF7C5FC07460B481838D0F8581270
:106790003846884704EBC402074901EBC201487838
:1067A00000F05EF8074604481838D0F8581238460A
:1067B0008847BDE8F08100007012002010B5042267
:1067C00000210846FFF7EEFE022204210020FFF719
:1067D000FAFE042206210120FFF7E4FE02220A212C
:1067E0000120FFF7F0FE04220C210220FFF7DAFE61
:1067F000022210211046FFF7E6FE04221221032098
:10680000FFF7D0FE022216210320FFF7DCFE042250
:1068100018211046FFF7C6FE02221C210420FFF7B4
:10682000D2FE04221E210520FFF7BCFE02222221F7
:106830000520FFF7C8FE042224210620FFF7B2FE40
:10684000022228210620FFF7BEFE04222A2107206B
:10685000FFF7A8FE02222E210720FFF7B4FE10BD8D
:1068600070B5054600260024372000F045F828467C
:1068700000F05CF8012211030B48FBF743F90FE02D
:106880000520FBF71FF8FFF72DFA0446102C00D067
:1068900007E03046711CCEB2C82801DDFA2070BD79
:1068A000EEE700BF2046FAE70004024070B5054657
:1068B00000260024362000F01FF8284600F036F8A5
:1068C000012211030B48FBF71DF90FE00520FAF731
:1068D000F9FFFFF707FA0446102C00D007E0304616
:1068E000711CCEB2C82801DDFA2070BDEEE700BFF2
:1068F0002046FAE70004024010B5044601221103C5
:106900000948FBF7FFF800224FF480510648FBF7D7
:10691000F9F8022000F000FC2046FFF782FC02207C
:1069200000F0FAFB10BD00000004024010B5044660
:106930002046FFF776FC10BD10B54FF48071054876
:10694000FBF7CEF808B9FFF757FB0349D1F860020F
:10695000804710BD000C02405812002038B5044694
:106960000CB9002038BD80488078002845D17E4889
:10697000C07884F820007C480179212001557A48AC
:1069800041792220015578488179232001557648A4
:10699000C179242001557448017A84F82510417A80
:1069A00084F82610817A84F82710C17A28200155AE
:1069B0006D48017B84F82910417B84F82A10817B83
:1069C00084F82B10C17B2C2001556748017C84F88A
:1069D0002D10417C84F82E10817C84F82F10C17C0E
:1069E000302001556048017D84F83110417D84F8E4
:1069F0003210817D84F8331037E004F13400FFF762
:106A000009F904F13800FFF7EDF804F13C00FFF755
:106A100019F956A0F9F7F4FC3720005D00903620F4
:106A2000035D3520025D94F834105DA0F9F7E8FCB1
:106A300094F83B00009094F83A3094F839203820CC
:106A4000015D5EA0F9F7DCFC94F83F00009094F83B
:106A50003E3094F83D203C20015D5FA0F9F7D0FC6A
:106A6000FFF792F80A20FAF72DFF617801EBC102D7
:106A70003D49183101EBC20048222146F9F715FFC4
:106A8000A07830B101281ED0022841D0032868D157
:106A900059E06078E11CFFF737FD60780221FFF7CD
:106AA0006DFD21896078FFF751FD61896078FFF7FE
:106AB0009BFD6078FFF72CFB05462B48D0F8581259
:106AC000284688474DE0FFF716FB6078E11CFFF78A
:106AD0001BFD60780321FFF751FD21896078FFF7E6
:106AE00035FD61896078FFF77FFD6078FFF710FB67
:106AF00005461D48D0F85812284688476078FFF7A9
:106B0000AFFE05461848D0F858122846884728E0B6
:106B100060780321FFF732FD61896078FFF764FD3B
:106B20006078FFF7F5FA05460F48D0F85812284666
:106B300088476078FFF7BAFE05460B48D0F8581230
:106B4000284688470DE060780121FFF717FD60783F
:106B5000FFF7DEFA05460448D0F858122846884761
:106B600000BF00BF0120FDE658120020BEB2CCAC31
:106B70004950D0C5CFA22E2E2E2E2E2E2E2E2E2EAA
:106B80002E2E2E2E2E2E2E2E2E2E2E2E2E2E2E2E25
:106B90002E2E2E2E2E2E2E2E2E2E2E0D0A000000E4
:106BA00049503A253032642E253032642E25303259
:106BB000642E253032640D0A00000000475749500A
:106BC0003A253032642E253032642E253032642E40
:106BD000253032640D0A00004D61736B3A25303266
:106BE000642E253032642E253032642E25303264F6
:106BF0000D0A000010B520480078092839D2DFE8D6
:106C000000F038050C131A20262C320000224FF415
:106C100080511A48FAF776FF2BE000224FF400610A
:106C20001648FAF76FFF24E000224FF400411448A1
:106C3000FAF768FF1DE0002280211148FAF762FF91
:106C400017E0002204210F48FAF75CFF11E0002250
:106C500001210C48FAF756FF0BE001229103084886
:106C6000FAF750FF05E0012210210748FAF74AFF22
:106C700000BF00BF10BD0000AC000020000C0240AF
:106C800000100240000402400008024010B5044613
:106C900002221A492046F9F778FD10B900F05EF893
:106CA0002BE0032216492046F9F76FFD10B900F0DA
:106CB00003F922E0032213492046F9F766FD10B9D3
:106CC00000F070F919E003220F492046F9F75DFD45
:106CD00010B900F073F810E003220C492046F9F7D0
:106CE00054FD10B900F06AF907E003220849204674
:106CF000F9F74BFD08B900F0C7F910BD5CA000081A
:106D000066A000086AA000086EA0000872A0000833
:106D100076A000083EB50D2009490A4A0A4BCDE984
:106D20000021029009A232210B48F9F775FB0A48AD
:106D3000F9F70CFDC4B22146074800F0BFFC3EBD88
:106D400059A000085CA0000846A000082573257320
:106D50002573256300000000380800200120044945
:106D6000487008460078062801D001200870704756
:106D70009C0800203EB50D2009490A4A0A4BCDE97E
:106D80000021029009A232210B48F9F745FB0A487D
:106D9000F9F7DCFCC4B22146074800F08FFC3EBD89
:106DA00059A000086EA0000846A0000825732573AE
:106DB00025732563000000003808002000B52DED84
:106DC000028B83B000200090019002909FED230A77
:106DD000B0EE408A22480068224A127881180A22BE
:106DE000684600F0E5FD012015E000BF1DF8001029
:106DF00030290ADB1DF80010392906DC1DF80010C7
:106E00003039C9B20DF8001002E000210DF8001071
:106E100000BF411CC8B20728E7DD0DF1010001F0F9
:106E200027FEB0EE408A9DF800002D2803D1B1EE78
:106E3000480AB0EE408A0C480078062802D00520A7
:106E4000094908709FED090A28EE000A064880EDFE
:106E5000010A03B0BDEC028B00BD00000000000081
:106E60006C000020700000209C08002000007A4484
:106E70003EB50D2009490A4A0A4BCDE9002102908E
:106E800009A232210B48F9F7C7FA0A48F9F75EFC64
:106E9000C4B22146074800F011FC3EBD59A00008CD
:106EA00066A0000846A00008257325732573256396
:106EB00000000000380800207CB500200090019000
:106EC00016480078401C15490870154800680A46A5
:106ED000127881180522684600F06AFD114C6D4653
:106EE0000522611C2846F9F750FC48B901200E49DB
:106EF000887008460078062805D00220087002E055
:106F000000200949887008480078012805D1064802
:106F1000807810B9012000F009F87CBD70000020D5
:106F20006C0000204BA000089C0800207FB50446A0
:106F300074B10D201249134A134BCDE90032CDE94B
:106F40000210124B12A232211448F9F765FA0DE033
:106F50000D200B49124A0C4BCDE90032CDE902104D
:106F60000A4B0BA232210D48F9F756FA0B48F9F7F4
:106F7000EDFBC5B22946094800F0A0FB7FBD00002B
:106F800059A000084BA000086AA0000846A000080D
:106F900025732573257325732563000038080020A9
:106FA00052A00008704710B5002000F031F810BD65
:106FB00010B5012000F02CF810BD00007CB50020B9
:106FC000009001900E480078401C0D4908700D4853
:106FD00000680A46127881180522684600F0E8FC2D
:106FE000094C6D460522611C2846F9F7CEFB18B9FD
:106FF00001200649C87002E000200449C8707CBD29
:10700000700000206C0000204BA000089C080020AD
:107010007FB5044674B10D201249134A134BCDE9D4
:107020000032CDE90210124B12A232211448F9F7B6
:10703000F3F90DE00D200B49124A0C4BCDE900325B
:10704000CDE902100A4B0BA232210D48F9F7E4F901
:107050000B48F9F77BFBC5B22946094800F02EFB27
:107060007FBD000059A000084BA0000876A00008D2
:1070700046A000082573257325732573256300003A
:107080003808002052A000080C480078022805D1DA
:1070900000200A49C870032008700EE007480078F5
:1070A000032805D101200549C8700420087004E0B8
:1070B00000200249C8700120087070479C08002019
:1070C00010B5012280210C48FAF71CFD01221103A2
:1070D0000A48FAF717FD0122D1020848FAF712FD13
:1070E000002240210448FAF70DFD00224FF4806190
:1070F0000248FAF707FD10BD000C024000080240EC
:1071000001B50098FAF7DEFB08BD00E000BF010002
:10711000A0F10100FAD1704711B526E0009CB4F54A
:10712000617F02D94FF4617400E0009C23464FF068
:10713000E024A069A82404FB1301002908DB00BF98
:107140004FF0E024A26982420CDA8A42F8DA09E0C0
:10715000084C214400BF4FF0E024A2698242FADDCE
:107160008A42F8DC009CE41A0094009C002CD5D1E3
:1071700018BD00004090020010B500F0ADFA4E4876
:10718000007800F0010204214C48FAF7BBFC4A48A1
:107190000078C0F3400208214848FAF7B3FC46489B
:1071A0000078C0F3800210214448FAF7ABFC424853
:1071B0000078C0F3C00220214048FAF7A3FC3E4803
:1071C0000078C0F3001240213C48FAF79BFC3A4893
:1071D0000078C0F340124FF400513948FAF792FC9E
:1071E00035480078C0F380124FF480413448FAF7F4
:1071F00089FC31480078C2094FF400413048FAF761
:1072000081FC30480078304908702B4880782D493F
:1072100008702D480078097888420AD02649887875
:1072200000F0A0F92449487800F09CF900F056F8E5
:1072300005E02149487800F095F900F04FF81E4824
:10724000C07800F0010020B11B48C078401E1A49E8
:10725000C8701948C078C0F3400020B11648C07803
:10726000801E1549C8701448C078C0F3800060B112
:1072700049F2187015490968486298201449086055
:107280000D48C078001F0C49C870FDF755FD000A75
:1072900010490870FDF750FD0E49487010210E4846
:1072A000FAF71EFC044620210B48FAF719FC04EB00
:1072B00040000849887010BDC0080020001002403E
:1072C0000008024009020020080200206803002094
:1072D00018000020CA0800200000024010B500225B
:1072E0004FF480710748FAF70DFC0A20FFF714FFEE
:1072F000012211020348FAF705FC0A20FFF70CFFF0
:1073000010BD00000008024010B5002415480068B8
:1073100020F00C001349086004E0601CC4B2012096
:10732000FFF7FAFE02210F48FAF7DAFB08B1C82C82
:10733000F3DBC82C01DB012010BD002404E0601C3D
:10734000C4B20120FFF7E8FE02210648FAF7C8FBA5
:1073500008B9F02CF3DBF02C01DB0120ECE7002076
:10736000EAE70000000802402DE9F04100F0A4F82F
:1073700000F082F8FFF7C8FFCC2000F0A9F8BE208B
:1073800000F0A6F800F066F8074600F063F805463E
:10739000072D05DDE843C5B2F843C7B2002600E07B
:1073A00001262C46200204B2E01904B200EE104A75
:1073B000B8EEC00AF6EE040A20EE200ABDEEC00ABE
:1073C00010EE100A04B216B12046BDE8F08160420A
:1073D00000B2FAE710B5012202210448FAF792FB45
:1073E00000F04AF8FFF790FF10BD000000080240CF
:1073F00010B51748006820F00C00154908600846D1
:10740000006840F004000860002202211048FAF7EA
:1074100079FB0220FFF780FE012202210C48FAF7D7
:1074200071FB0B48006820F00C00094908600C2033
:10743000FFF772FE02210648FAF752FB08B1012459
:1074400000E000243220FFF767FE204610BD000058
:107450000008024070B50026012508E0FFF7C8FFCC
:107460000446E00140EA6600C6B2681CC5B2082DB9
:10747000F4DD304670BD000010B50E48006820F005
:107480000C000C4908600846006840F004000860E1
:10749000002202210748FAF735FB40F2EE20FFF701
:1074A0003BFE012202210348FAF72CFB0F20FFF7D5
:1074B00033FE10BD0008024010B5FFF7DDFFFFF7F7
:1074C00023FFCC2000F004F8442000F001F810BDA8
:1074D00070B504461B48006820F00C00194908608C
:1074E0000846006840F004000860012526E004F02A
:1074F0000106641086B1002202211248FAF702FB4D
:107500000220FFF709FE012202210E48FAF7FAFADB
:107510003C20FFF701FE0FE0002202210948FAF7A4
:10752000F1FA3C20FFF7F8FD012202210548FAF7A5
:10753000E9FA0220FFF7F0FD681CC5B2082DD6DD80
:1075400070BD00000008024013B50C464FF6FF73F3
:10755000012269460248FCF703FA00981CBD0000AE
:107560008804002070B504462546002628E0002245
:107570004FF400411448FAF7C5FA05F0800028B12D
:10758000012240211148FAF7BDFA04E0002240210F
:107590000E48FAF7B7FA6806050E00224FF40041CC
:1075A0000948FAF7AFFA0A20FFF7B6FD0122D10326
:1075B0000548FAF7A7FA0A20FFF7AEFD701CC6B21D
:1075C000082ED4DB70BD0000000C02400000024019
:1075D00038B504460D46002000901649087016483C
:1075E000046008460078001D08701448407870B99F
:1075F000114800680A46127881180222684600F095
:10760000D7F90C480078801C0A4908700DE00A4838
:107610000068084A127881180322684600F0C8F909
:1076200004480078C01C034908706846FFF72EFB29
:1076300038BD0000700000206C0000209C08002075
:1076400010B519480078252802D101201749086093
:1076500016480068012821D1134800781449154ABA
:107660001268885413480068401C12490860084694
:107670000068401E0E49085C2A280FD10D4800689A
:10768000801E085C2A2809D10A4801780848FFF7BB
:107690009FFF002007490860044908600122024951
:1076A0000548FCF733F910BD710000207800002078
:1076B0006A080020740000201805002070B50446F8
:1076C0000D4603482A46214683680248984770BD04
:1076D0009C0800201805002010B50A480068012801
:1076E0000ED100200749086002210748FAF700FA86
:1076F000FFF73AFE05490880084600880449C88417
:1077000010BD000000020020001002400A0200200C
:10771000D6080020FAF73AFBFCF710FE4FF47A7017
:10772000FFF7EEFCFCF752FAFCF7FCF9FCF7C2F9A4
:10773000FCF74AFBFCF766FBFCF786FBFCF726FC34
:10774000FCF740FCFCF75AFCFCF774FCFCF78EFCE1
:10775000FCF7D0FBFCF7F4FB8748FBF72BFA3C2146
:107760008648FBF7FFFA49F21870844909684862B5
:10777000FDF77EFBFDF7C8FFC820FFF7C1FCFDF752
:1077800017FDC820FFF7BCFCFFF79AFCC820FFF7E5
:10779000B7FC01F0D1F9FFF71DFEFDF7BFFA00F0CD
:1077A000B1FAC820FFF7ACFCFEF77EFBFEF7ECFB5E
:1077B000E0E0FFF7C1F87248008800EE100AB8EE6A
:1077C000400ADFED700A80EE201A6F4890ED000A43
:1077D000B4EE401AF1EE10FA23D16948408800EE69
:1077E000100AB8EE400ADFED670A80EE201A6748FB
:1077F00090ED000AB4EE401AF1EE10FA11D1604893
:10780000808800EE100AB8EE400ADFED5E0A80EED6
:10781000201A5F4890ED000AB4EE401AF1EE10FA1B
:107820005FD05748008800EE100AB8EE400ADFED3E
:10783000550A80EE201A544880ED001A50484088BE
:1078400000EE100AB8EE400ADFED4E0A80EE201A74
:107850004E4880ED001A4A48808800EE100AB8EEC3
:10786000400ADFED480A80EE201A494880ED001AF0
:10787000454890ED000AF3EE090AB4EEE00AF1EE95
:1078800010FA03DDB3EE090A80ED000A3F4890EDDF
:10789000000AF3EE090AB4EEE00AF1EE10FA03DD95
:1078A000B3EE090A80ED000A394890ED000AF3EEC4
:1078B000090AB4EEE00AF1EE10FA03DDB3EE090AAC
:1078C00080ED000A304890ED000AFDF7FFFF2F48D9
:1078D00090ED000AFDF7AEFF2D4890ED000AFDF790
:1078E000CFFF2C48006820B101F09EF90020294903
:1078F0000860FDF7BFFAFDF757FDFDF787FAFFF7C0
:107900003BFC25480068254908601C480068406A1F
:10791000214908600846006820490968401A204942
:10792000884205DA1F480068401C1E4908600DE0C7
:107930001948006819490968401A4CF250318842C8
:1079400004DD18480068401E1649086015480068A4
:10795000C0EB004010490968084413490860084614
:1079600000684FF6FF7101EA1040104908850E4883
:10797000008848851DE70000B00300206803002050
:10798000CE00002000007A44000000200400002007
:1079900008000020E0010020100000200C00002062
:1079A000B03CFFFF1800002014000020D608002083
:1079B00010B503E011F8013B00F8013B1300A2F100
:1079C0000104A2B2F6D110BD2DE9F04104460D46E6
:1079D0000CB1022D01DABDE8F08126786778012E1E
:1079E00001D0002E48D1052F3AD008DC012F0DD050
:1079F000022F11D0032F15D0042F37D118E0062FF6
:107A00001CD00F2F20D0102F30D123E0A81E81B220
:107A1000A01C00F0E1F92EE0A81E81B2A01C00F02D
:107A200057FB28E0A81E81B2A01C00F0C5FC22E094
:107A3000A81E81B2A01C00F0EDFD1CE0A81E81B2C2
:107A4000A01C01F0ADFD16E0A81E81B2A01C01F043
:107A50000FFA10E0A81E81B2A01C01F091FB0AE011
:107A6000A81E81B2A01C01F0B7FC04E060780121DF
:107A700000F078F800BF00BF00BFACE72DE9F0418F
:107A800004460D460CB1022D01DABDE8F08100205C
:107A900003E0215C324A1154401C0428F9DBA6792A
:107AA000E779012E01D0002E58D1052F48D008DCEF
:107AB000012F0DD0022F13D0032F19D0042F47D13F
:107AC0001EE0062F24D00F2F2AD0102F40D12FE0F8
:107AD000A5F1080081B204F1080000F02FFA3CE0A3
:107AE000A5F1080081B204F1080000F09FFB34E02A
:107AF000A5F1080081B204F1080000F0E3FC2CE0DD
:107B0000A5F1080081B204F1080000F005FE24E0B0
:107B1000A5F1080081B204F1080001F0A1FD1CE00C
:107B2000A5F1080081B204F1080001F057FA14E051
:107B3000A5F1080081B204F1080001F0A9FB0CE0F6
:107B4000A5F1080081B204F1080001F0ABFC04E0EB
:107B5000E079012100F042F800BF00BF00BF94E7C8
:107B600092010020F0B5ADF2044D05460E4600240A
:107B7000002701222146641C01A8425445F08002DE
:107B80002146641C42542146641C46542146FCF79D
:107B90009BFA07462146641C01A847543A12214625
:107BA000641C42540B48008AA04201DB204601E0DD
:107BB0000848008A074948824A8AC86801A9F8F734
:107BC0002FFE0448428AC168034800F089FF0DF285
:107BD000044DF0BD241C00208804002070B5ADF5D4
:107BE000806D05460E460024234802782146641C19
:107BF0000DF8012042782146641C0DF8012082789E
:107C00002146641C0DF80120C2782146641C0DF841
:107C1000012000222146641C0DF801200322214688
:107C2000641C0DF8012001222146641C0DF801207E
:107C300045F080022146601CC4B20DF801202046A8
:107C4000611CCCB20DF80060FF2C01DC214600E085
:107C5000FF210A48816201468A6A486A6946F8F744
:107C6000DFFD0648008D82B20448416A0020FEF71D
:107C700019FC0DF5806D70BD920100205812002096
:107C80002DE9F041002414480568C488022C01DA6B
:107C9000BDE8F081042211492846F8F72BFD20B9F0
:107CA0002146284600F0DCFDF2E7A01E295C601E9C
:107CB000285C41EA0027A01E81B22846FCF704FA9E
:107CC0000646B74200D0E3E7034AD1881068FFF7C1
:107CD0007BFE00BFDCE70000241C00208E0100209A
:107CE00070B500240648056B808E84B2022C00DA41
:107CF00070BD21462846FFF7C1FE00BFF8E700002F
:107D00005812002010B50E480E49086000208880E7
:107D1000C88008720C48C8604FF480600882002058
:107D20004882012209490A48FBF7F0FD6FF0010083
:107D30000849096808610748FAF73CFF10BD0000D0
:107D4000560A0020241C0020560E00200C020020A1
:107D500088040020F803002010B51848808840F2FD
:107D6000FF3188420EDB00201449888008460068F5
:107D7000002101604FF6FF730A2211A11348FBF79F
:107D8000EFFD14E0124801780C4882888088401C7E
:107D90000A4B98801846006881540E48FAF75EFF37
:107DA00000200C49096848620A48FAF703FF0122DB
:107DB00007490648FBF7AAFD10BD0000241C00205F
:107DC000CAFDBEDDD2E7B3F6000000008804002043
:107DD0000C020020F80300202DE9F04FADF2144D05
:107DE000054600240020CDF804044FF4806101A86A
:107DF000F8F78DFD6878297840EA0129E878A978B4
:107E000040EA0126012E01DA502E70DCB9F15F0F35
:107E10006EDC06EB090060287EDCF01DC11700EB6C
:107E20005171C1F3C701CDF8101401222046611C25
:107E3000CCB201A90A542046611CCCB201A90A5453
:107E40002046621CD4B201AADDF810141154002798
:107E5000BB462FE0002001A9085582461BE009EB34
:107E6000070188B20DF20C41F9F7C6F801A8005DD0
:107E70009DF80C1401FA0AF1084301A90855781C71
:107E800087B2B74203DB0120CDF8040406E00AF113
:107E9000010000F0FF0ABAF1080FE0DB00BF601C30
:107EA000C4B2DDF80404012800D107E00BF10100A1
:107EB00000F0FF0BDDF810048345CBDB00BF21464B
:107EC00001A8FCF701F980462046611CCCB201A94B
:107ED00001F800804FEA28222046611CCCB201A99B
:107EE0000A541448008AA04203DB204603E017E04E
:107EF00012E01048008A0F4948824A8AC86801A9DE
:107F0000F8F78EFC0B48428AC1680B4800F0E8FD88
:107F10000DF2144DBDE8F08F0220CDF8080402E008
:107F20000320CDF808040120DDF80814FFF71AFE3D
:107F300000BFEDE7241C0020880400202DE9F04F4D
:107F4000ADF20C4D054600240020CDF800044FF49E
:107F500080616846F8F7DBFC6878297840EA0129F7
:107F6000E878A97840EA0126012E01DA502E7ADC61
:107F7000B9F15F0F78DC06EB09006028FADCF01D30
:107F8000C11700EB5171C1F3C7074F480278204673
:107F9000611CCCB20DF800204B4842782146601C91
:107FA000C4B20DF80120484882782046611CCCB24A
:107FB0000DF800204448C2782046611CCCB20DF870
:107FC0000020F81C02122046611CCCB20DF80020E3
:107FD000F81CC2B22046611CCCB20DF80020012270
:107FE0002046611CCCB20DF800202046611CCCB2AA
:107FF0000DF800202046611CCCB20DF800704FF047
:1080000000084FF0000A34E000200DF80400834619
:108010001EE009EB080188B20DF58161F8F7ECFF6D
:108020001DF804009DF8081401FA0BF10843C0B2D2
:108030000DF8040008F101001FFA80F8B04503DBD9
:108040000120CDF8000406E00BF1010000F0FF0B69
:10805000BBF1080FDDDB00BF601CC4B2DDF800041B
:10806000012802D107E024E01FE00AF1010000F03E
:10807000FF0ABA45C8DB00BFFF2C01DC214600E047
:10808000FF211248816201468A6A486A6946F8F708
:10809000C7FB0E48008D82B20C48416A0020FEF7F3
:1080A00001FA0DF20C4DBDE8F08F0220CDF804046A
:1080B00002E00320CDF804040120DDF80414FFF7EA
:1080C0008DFD00BFEDE70000920100205812002056
:1080D0002DE9F04FADF2144D054600240020CDF8F7
:1080E00004046878297840EA0129E878A97840EA08
:1080F0000126012E01DA602E71DCB9F15F0F6FDC11
:1081000006EB090060287FDCF01DC11700EB517100
:10811000C1F3C701CDF8101401222046611CCCB276
:1081200001A90A5402222046611CCCB201A90A54BA
:108130002046621CD4B201AADDF8101411540027A5
:10814000BB462FE0002001A9085582461BE009EB41
:10815000070188B20DF20C41F8F76AFF01A8005D33
:108160009DF80C1401FA0AF1084301A90855781C7E
:1081700087B2B74203DB0120CDF8040406E00AF120
:10818000010000F0FF0ABAF1080FE0DB00BF601C3D
:10819000C4B2DDF80404012800D107E00BF10100AE
:1081A00000F0FF0BDDF810048345CBDB00BF214658
:1081B00001A8FBF789FF80462046611CCCB201A9CB
:1081C00001F800804FEA28222046611CCCB201A9A8
:1081D0000A541448008AA04203DB204603E017E05B
:1081E00012E01048008A0F4948824A8AC86801A9EB
:1081F000F8F716FB0B48428AC1680B4800F070FC88
:108200000DF2144DBDE8F08F0220CDF8080402E015
:108210000320CDF808040220DDF80814FFF7A2FCC3
:1082200000BFEDE7241C0020880400202DE9F04F5A
:10823000ADF20C4D054600240020CDF8000468780E
:10824000297840EA0129E878A97840EA0126012E38
:1082500001DA602E7BDCB9F15F0F79DC06EB0900F7
:108260006028FADCF01DC11700EB5171C1F3C7079C
:108270004F4802782046611CCCB20DF800204C48D3
:1082800042782146601CC4B20DF80120484882782B
:108290002046611CCCB20DF800204548C27820462B
:1082A000611CCCB20DF80020F81C02122046611CA3
:1082B000CCB20DF80020F81CC2B22046611CCCB232
:1082C0000DF8002001222046611CCCB20DF80020E0
:1082D00002222046611CCCB20DF800202046611C11
:1082E000CCB20DF800704FF000084FF0000A34E0F7
:1082F00000200DF8040083461EE009EB080188B257
:108300000DF58161F8F794FE1DF804009DF808143E
:1083100001FA0BF10843C0B20DF8040008F10100A6
:108320001FFA80F8B04503DB0120CDF8000406E019
:108330000BF1010000F0FF0BBBF1080FDDDB00BF0C
:10834000601CC4B2DDF80004012802D107E024E07B
:108350001FE00AF1010000F0FF0ABA45C8DB00BFC8
:10836000FF2C01DC214600E0FF211248816201461A
:108370008A6A486A6946F8F753FA0E48008D82B255
:108380000C48416A0020FEF78DF80DF20C4DBDE857
:10839000F08F0220CDF8040402E00320CDF804049D
:1083A0000220DDF80414FFF719FC00BFEDE7000020
:1083B00092010020581200202DE9F04FADF2044D3B
:1083C000064600241EB90DF2044DBDE8F08F70780A
:1083D000317840EA0127F078B17840EA0125012D93
:1083E00063DB602D61DC5F2F5CDC7819002859DBD2
:1083F0007819602856DC01222046611CCCB201A904
:108400000A5403222046611CCCB201A90A54680612
:10841000020E2046611CCCB201A90A544FF000089C
:1084200016E007EB080188B2F8F7D2FD81464FEA63
:1084300029222046611CCCB201A90A542046611CA5
:10844000CCB201A901F8009008F101001FFA80F8F0
:10845000A845E6DB214601A8FBF736FE824620460A
:10846000611CCCB201A901F800A04FEA2A222046E3
:10847000611CCCB201A90A541048008AA04201DB59
:10848000204601E00D48008A0C4948824A8AC868A3
:1084900001A9F8F7C5F90948428AC168084800F0FF
:1084A0001FFB90E74FF0020B01E04FF0030B594622
:1084B0000320FFF757FB00BF85E70000241C0020C6
:1084C000880400202DE9F04FADF2044D06468A469F
:1084D00000241EB90DF2044DBDE8F08F707831789C
:1084E00040EA0127F078B17840EA0125012D7DDBD3
:1084F000602D7BDC5F2F7EDC781900287BDB781910
:10850000602878DC414802782046611CCCB201A981
:108510000A543E4842782046611CCCB201A90A5454
:108520003A4882782046611CCCB201A90A543748E7
:10853000C2782046611CCCB201A90A54022000EB8B
:108540004500401CC0F307222046611CCCB201A9A3
:108550000A54022000EB4500401CC2B22046611CB8
:10856000CCB201A90A5401222046611CCCB201A957
:108570000A5403222046611CCCB201A90A546806A1
:10858000020E2046611CCCB201A90A544FF000082B
:1085900016E007EB080188B2F8F71AFD81464FEAAA
:1085A00029222046611CCCB201A90A542046611C34
:1085B000CCB201A901F8009008F101001FFA80F87F
:1085C000A845E6DBFF2C01DC214600E0FF21104836
:1085D000816201468A6A486A01A9F8F721F90C48C4
:1085E000008D82B20A48416A002001E006E002E004
:1085F000FDF758FF6EE74FF0020B01E04FF0030B61
:1086000059460320FFF7EAFA00BF63E79201002012
:10861000581200202DE9F04FADF2044D054600241C
:108620001DB90DF2044DBDE8F08F6878297840EA55
:108630000127E878A97840EA0126012E60DB602E48
:108640005EDC5F2F59DCB819602856DC0122204619
:10865000611CCCB201A90A5404222046611CCCB290
:1086600001A90A547006020E2046611CCCB201A971
:108670000A544FF0000816E007EB080188B2F8F73B
:10868000B1FC81464FEA29222046611CCCB201A9E7
:108690000A542146601CC4B201A800F8019008F1F8
:1086A00001001FFA80F8B045E6DB214601A8FBF780
:1086B0000BFD82462046611CCCB201A901F800A046
:1086C0004FEA2A222046611CCCB201A90A54104864
:1086D000008AA04201DB204601E00D48008A0C49D7
:1086E00048824A8AC86801A9F8F79AF80848428A75
:1086F000C168084800F0F4F993E74FF0020B01E07D
:108700004FF0030B59460420FFF72CFA00BF88E70F
:10871000241C0020880400202DE9F04FADF2044D08
:1087200006468A4600241EB90DF2044DBDE8F08FBE
:108730007078317840EA0127F078B17840EA012575
:10874000012D7CDB602D7FDC5F2F7ADC78196028BF
:1087500077DC414802782046611CCCB201A90A545A
:108760003D4842782146601CC4B201A842543A48B0
:1087700082782046611CCCB201A90A543648C278DE
:108780002046611CCCB201A90A54022000EB45002E
:10879000401CC0F307222046611CCCB201A90A5438
:1087A000022000EB4500401CC2B22046611CCCB246
:1087B00001A90A5401222046611CCCB201A90A5425
:1087C00004222046611CCCB201A90A546806020E9C
:1087D0002046611CCCB201A90A544FF0000816E0F3
:1087E00007EB080188B2F8F7FDFB81464FEA292222
:1087F0002146601CC4B201A842542046611CCCB280
:1088000001A901F8009008F101001FFA80F8A845BD
:10881000E6DBFF2C01DC214600E0FF210F488162EE
:1088200001468A6A486A01A9F7F7FAFF0B48008DEA
:1088300082B20A48416A0020FDF734FE74E703E083
:10884000FFE74FF0020B01E04FF0030B5946042005
:10885000FFF7C4F900BF67E792010020581200201B
:1088600070B504460D4600200DE0011D615C0C4A08
:10887000115400F10801615C0A4A1154011D615C48
:10888000094A1154401C0428EFDBE0790A300649FC
:10889000C870022005498870FDF776FB70BD0000A6
:1088A0009C010020A4010020A001002058120020FB
:1088B00010B5012211031448F9F724F90122D1025D
:1088C0001148F9F71FF90122D1031048F9F71AF9F5
:1088D00000224FF480410D48F9F714F9012280215C
:1088E0000A48F9F70FF9012204210948F9F70AF9B2
:1088F000012211460648F9F705F900221021054822
:10890000F9F700F910BD0000000C02400010024011
:10891000000402400008024001B582B04FF47A70B2
:10892000012301AA02A900900248F9F737FF9DF838
:1089300004000EBD100300203D480068401C3C4967
:10894000086008460068042805DD012039490860F0
:1089500000203749086038480068401C36490860E4
:1089600008460068092805DD012034490860002018
:108970003149086032480068401C314908600846A7
:108980000068182805DD01202E49086000202C49C8
:1089900008602D480068401C2B49086008460068A4
:1089A000312805DD0120294908600020264908609A
:1089B00027480068401C264908600846006863286C
:1089C00005DD012023490860002021490860224874
:1089D0000068401C2049086008460068B0F5967F92
:1089E00005DB01201D49086000201B4908601C4868
:1089F0000068401C1A49086008460068B0F5FA7F14
:108A000005DB012017490860002015490860164859
:108A10000068401C1449086008460068B0F57A7F79
:108A200005DB01201149086000200F4908607047EC
:108A3000CC010020C8010020D4010020D00100207A
:108A4000DC010020D8010020E4010020E00100202A
:108A5000EC010020E8010020F4010020F0010020DA
:108A6000FC010020F8010020040200200002002088
:108A70000178194A5143427840F6354312FB03F21C
:108A800001EB4211827840F2712312FB03F201EBF9
:108A90000211C27802EB4203C3EBC21201EBC20126
:108AA000027902EBC20303EB021201EB820142796D
:108AB00002EB820201EB42018279114400EE901A2E
:108AC000B0EE601AB8EEC11ADFED041A81EE212A69
:108AD000B0EE420A7047000040420F000050C3470A
:108AE00070B504460D461646324629462046FAF72A
:108AF00097FF70BD70B50446FEF77CF88020FBF749
:108B0000E7FB2046FBF7E4FBFBF748FB0546FFF7D6
:108B1000CFFE284670BD70B505460C46FEF76AF8D4
:108B20000020FBF7D5FB2846FBF7D2FB2046FBF7DE
:108B3000CFFBFFF7BDFE70BD10B5FFF7B9FE0022F9
:108B40004FF400713648F8F7DDFF0A20FEF7D8FA37
:108B500001203449087001210020FFF7DCFF0A20C2
:108B6000FEF7CEFA08213020FFF7D5FF02202D496D
:108B7000087001210020FFF7CEFF0A20FEF7C0FA9F
:108B800008213020FFF7C7FF032026490870012184
:108B90000020FFF7C0FF0A20FEF7B2FA08213020BC
:108BA000FFF7B9FF012251021D48F8F7ABFF0A2079
:108BB000FEF7A6FA04201B49087001210020FFF7E8
:108BC000AAFF0A20FEF79CFA08213020FFF7A3FF36
:108BD00005201449087001210020FFF79CFF0A209E
:108BE000FEF78EFA08213020FFF795FF06200D4989
:108BF000087001210020FFF78EFF0A20FEF780FA9F
:108C000008213020FFF787FF012006490870002265
:108C100041020348F8F776FF0A20FEF771FA10BD0B
:108C200000080240AC00002010B52DED048B7F48F9
:108C30000078002869D001207D49087060E07C48F8
:108C40000078032805DD012251027A48F8F75AFF1F
:108C500005E000224FF400717648F8F753FF092031
:108C6000FFF748FF7449C8700A20FFF743FF7249B5
:108C700008710846C07871490860714800680002B0
:108C800008606D480079096808436C490860084627
:108C90000068B0F5004F13DD09686A4A881A00F0D1
:108CA000B8FF41EC190B9FED680B53EC102B00F053
:108CB0002BFE41EC180B00F04DFD6549086013E0F8
:108CC0005E490968A1F59A7000F0A3FF41EC190B09
:108CD0009FED5D0B53EC102B00F016FE41EC180BD2
:108CE00000F038FD5A4908600020504908700921F9
:108CF0003020FFF710FF4E480078401C4C490870A8
:108D00004B48007807289ADB8DE00120484908701D
:108D100084E047480078032805DD012251024548D8
:108D2000F8F7F0FE05E000224FF400714148F8F733
:108D3000E9FE0620FFF7DEFE3F4908700720FFF737
:108D4000D9FE3D4948700820FFF7D4FE3A498870A3
:108D5000084600783F49086008460068000208603D
:108D600035484078096808433A4908600846006871
:108D70000002086030488078096808433549086077
:108D800008460068B0F5000F0FDB08460068A0F148
:108D9000807000EE100AB8EEC00ADFED2F0A80EEF8
:108DA000201A2E4880ED001A0BE02A4890ED000AA8
:108DB000B8EEC00ADFED280A80EE201A274880EDC1
:108DC000001A2648D0ED000A9FED250A9FED251ACE
:108DD00001EE200AF2EE080A80EE201A224880ED09
:108DE000001A90ED000AF2EE040A20EE200ABCEE12
:108DF000C00A10EE100A81B21C4A0D4800780C30EF
:108E000022F8101001200949087008213020FFF7CE
:108E100082FE07480078401C054908700448007825
:108E20000728FFF676AFBDEC048B10BDCC00002008
:108E3000AC00002000080240AD000020C800002067
:108E4000B400002034010100000000000000704068
:108E5000BC000020C40000200000004BC000002027
:108E600000A00C4600401C46B8000020D608002098
:108E70002DE9F04FADF2144D044600250020CDF849
:108E800004046078217840EA012AE078A17840EA79
:108E900001262079CDF80C04012E77DB502E75DCED
:108EA000DDF80C04C000B042F7DBBAF15F0F6EDCF6
:108EB0000AEB060060287EDC0027A94636E009F1AF
:108EC0000500205CCDF808044FF0000B21E00120E4
:108ED00000FA0BF0DDF80814084020B14FF47F4091
:108EE000CDF8100402E00020CDF810040AEB0701D1
:108EF00088B2DDF81014FBF7D5FE781C87B2B742B4
:108F000003DB0120CDF8040406E00BF1010000F0C2
:108F1000FF0BBBF1080FDADB00BFDDF8040401280A
:108F200000D107E009F1010000F0FF09DDF80C04B1
:108F30008145C4DB00BF01222846691CCDB20DF873
:108F400000200F222846691CCDB20DF800200DEB41
:108F5000050021680160281DC5B229466846FBF757
:108F6000B3F8804608F0FF022846691CCDB20DF820
:108F700000204FEA28222846691CCDB20DF80020B7
:108F80001448008AA84203DB284603E017E012E0F9
:108F90001048008A0F4948824A8AC8686946F7F72C
:108FA0003FFC0C48428AC1680B48FFF799FD0DF25F
:108FB000144DBDE8F08F0220CDF8000402E003203C
:108FC000CDF800040F20DDF80014FEF7CBFD00BF44
:108FD000EDE70000241C0020880400202DE9F04F5C
:108FE000ADF2144D0546894600240020CDF8040456
:108FF0006878297840EA012BE878A97840EA0126C8
:109000002879CDF80C04012E7EDB502E7CDCDDF8B7
:109010000C04C000B042F7DBBBF15F0F75DC0BEB5B
:1090200006006028FADC0027A04636E008F10500BB
:10903000285CCDF808044FF0000A21E0012000FA76
:109040000AF0DDF80814084020B14FF47F40CDF855
:10905000100402E00020CDF810040BEB070188B2E9
:10906000DDF81014FBF71EFE781C87B2B74203DB55
:109070000120CDF8040406E00AF1010000F0FF0A27
:10908000BAF1080FDADB00BFDDF80404012800D1D3
:1090900007E008F1010000F0FF08DDF80C0480454E
:1090A000C4DB00BF344802782146601CC4B20DF80E
:1090B0000120314842782046611CCCB20DF80020D6
:1090C0002D4882782046611CCCB20DF800202A4839
:1090D000C2782046611CCCB20DF8002009F10200D4
:1090E000C0F307222046611CCCB20DF8002009F124
:1090F0000200C2B22046611CCCB20DF80020012251
:109100002046611CCCB201E02BE026E00DF80020E7
:109110000F222046611CCCB20DF800200DEB04009C
:1091200029680160201DC4B2FF2C01DC214600E04B
:10913000FF211248816201468A6A486A6946F7F748
:109140006FFB0E48008D82B20C48416A0020FDF78B
:10915000A9F90DF2144DBDE8F08F0220CDF80004FE
:1091600002E00320CDF800040F20DDF80014FEF724
:1091700035FD00BFEDE700009201002058120020ED
:109180002DE9F04FADF2044D044600261CB90DF256
:10919000044DBDE8F08F6078217840EA0128E0783E
:1091A000A17840EA012794F804A0012F62DB602F28
:1091B00060DCBAEB470F5DD1B8F15F0F57DC08EB0D
:1091C0000700602853DC002514E0062000EB450072
:1091D000205C052101EB4501615C40EA0120CDF8EE
:1091E000000408EB050188B2DDF80014FBF752FD1E
:1091F000681C85B2BD42E8DB01223046711CCEB24C
:109200000DF8002010223046711CCEB20DF800205F
:109210000DEB060021680160301DC6B2314668467C
:10922000FAF752FF814609F0FF023046711CCEB2B8
:109230000DF800204FEA29223046711CCEB20DF8FD
:1092400000201148008AB04201DB304601E00E48A0
:10925000008A0D4948824A8AC8686946F7F7E0FAE9
:109260000948428AC1680948FFF73AFC8FE74FF086
:10927000020B01E04FF0030B0BF0FF011020FEF793
:1092800071FC00BF83E70000241C0020880400203C
:109290002DE9F04FADF2044D0546894600241DB975
:1092A0000DF2044DBDE8F08F6878297840EA012876
:1092B000E878A97840EA012795F804A0012F7EDB21
:1092C000602F7CDCBAEB470F79D1B8F15F0F73DC0C
:1092D00008EB070060286FDC002614E0062000EB96
:1092E0004600285C052101EB4601695C40EA01204B
:1092F000CDF8000408EB060188B2DDF80014FBF796
:10930000C9FC701C86B2BE42E8DB314802782046B8
:10931000611CCCB20DF800202D4842782046611C1B
:10932000CCB20DF800202A4882782046611CCCB2CD
:109330000DF800202648C2782046611CCCB20DF8FA
:10934000002009F10200C0F307222046611CCCB2C4
:109350000DF8002009F10200C2B22046611CCCB217
:109360000DF8002001222046611CCCB20DF800202F
:1093700010222046611CCCB20DF800200DEB040039
:1093800029680160201DC4B2FF2C01DC214600E0E9
:10939000FF211048816201468A6A486A6946F7F7E8
:1093A0003FFA0C48008D82B20A48416A0020FDF75E
:1093B00079F875E703E0FFE74FF0020B01E04FF0AB
:1093C000030B0BF0FF011020FEF708FC00BF67E75E
:1093D00092010020581200202DE9F047ADF5806D74
:1093E00005468A4600246878297840EA0129E87809
:1093F000A97840EA012717B1B7F57F4F45D1B9F1F8
:109400005F0F3FDC39464846FBF74CFC0122204603
:10941000611CCCB20DF8002005222046611CCCB2A4
:109420000DF800200DEB040029680160201DC4B276
:1094300021466846FAF748FE0646F2B22046611C0D
:10944000CCB20DF8002032122046611CCCB20DF8CF
:1094500000201248008AA04201DB204601E00F48AC
:10946000008A0E4948824A8AC8686946F7F7D8F9DF
:109470000A48428AC1680A48FFF732FB0DF5806D41
:10948000BDE8F0874FF0020801E04FF003084146C5
:109490000520FEF767FB00BFF0E70000241C00205A
:1094A000880400202DE9F043ADF2044D05460E4638
:1094B00000246878297840EA0129E878A97840EA08
:1094C000012717B1B7F57F4F5ED1B9F15F0F58DCB7
:1094D00039464846FBF7E6FB2F4802782046611CD8
:1094E000CCB201A90A542C4842782046611CCCB267
:1094F00001A90A54284882782046611CCCB201A9EF
:109500000A542548C2782046611CCCB201A90A54ED
:10951000B01CC0F307222046611CCCB201A90A543A
:10952000B01CC2B22046611CCCB201A90A5401226F
:109530002046611CCCB201A90A5405222146601CB8
:10954000C4B201A84254204429680160201DC4B25D
:10955000FF2C01DC214600E0FF211048816201461A
:109560008A6A486A01A9F7F75BF90C48008D82B254
:109570000A48416A0020FCF795FF0DF2044DBDE852
:10958000F0834FF0020801E04FF003084146052048
:10959000FEF724FB00BFF0E79201002058120020E4
:1095A0002DE9F047ADF5806D05468A4600241DB9CA
:1095B0000DF5806DBDE8F0876878297840EA0127CD
:1095C000E878A97840EA01285F2F3CDC414638461C
:1095D000FBF760FB01222046611CCCB20DF8002095
:1095E00006222046611CCCB20DF800200DEB0400D1
:1095F00029680160201DC4B221466846FAF764FD5F
:109600000646F2B22046611CCCB20DF800203212A0
:109610002046611CCCB20DF800200F48008AA04201
:1096200001DB204601E00C48008A0B4948824A8A47
:10963000C8686946F7F7F4F80748428AC1680748DE
:10964000FFF74EFAB4E74FF0020949460620FEF74D
:1096500089FA00BFACE70000241C00208804002029
:109660002DE9F043ADF2044D05460E4600241DB928
:109670000DF2044DBDE8F0836878297840EA0127AF
:10968000E878A97840EA01285F2F56DC4146384641
:10969000FBF700FB2D4802782046611CCCB201A9E3
:1096A0000A542A4842782146601CC4B201A8425498
:1096B000264882782046611CCCB201A90A5423486E
:1096C000C2782046611CCCB201A90A54B01CC0F378
:1096D00007222046611CCCB201A90A54B01CC2B2B8
:1096E0002046611CCCB201A90A5401222046611C0B
:1096F000CCB201A90A5406222046611CCCB201A9B1
:109700000A5401A8204429680160201DC4B2FF2C1E
:1097100001DC214600E0FF210D48816201468A6A92
:10972000486A01A9F7F77CF80948008D82B2084819
:10973000416A0020FCF7B6FE9AE74FF0020949465D
:109740000620FEF74BFA00BF92E7000092010020CE
:109750005812002021F00042A2F16052B2F5801FA1
:1097600001F0004328BFD2F17F6C0BD95FEA001CE7
:1097700043EAC20242EB507018BF704728BF20F086
:1097800001007047B2F5801FBCBF184670474FEA12
:10979000410C1CF5001F02D2084600F03EBC70B51B
:1097A00000F0F8FA00000089FFF7F6BF4FF0004024
:1097B000A0F580007047000010B591EA030F48BF84
:1097C00083F0004300F14283841A71EB030C05D24D
:1097D000121943EB0C03001B61EB0C01DFF824E1D1
:1097E0004FEA1154A4EB135C1EEA430F18BF9EEA24
:1097F000445F73D023EA0E03DCF1200E21EA04510A
:1098000043F4801332D322FA0CFE10EB0E0023FA3D
:109810000CFE41EB0E01CCF1200E03FA0EFE10EB14
:109820000E0051F10001B1F5801FCCF1200E32D2B3
:1098300001EB045112FA0EF2BDE8104058BF704718
:10984000401C38BF5FEA420218BF7047002814BFAF
:1098500020F0010041F100014FEA410313F5001F20
:1098600038BF7047A1F1C04100F0E2BA012A43EBD2
:109870000302ACF1200CDCF11F0E32BF4FF0000EE2
:1098800023FA0CF310EB030041EB0451B4EB115F2E
:10989000D0D0A1EB045101F5801149085FEA3000F6
:1098A00001EB04510ED350F1000038BF12FA0EFE46
:1098B00008D1BDE81040C9E7401C38BF5FEA42024A
:1098C000CAD1C3E7BDE810404FEA410313F5001FBA
:1098D00038BF7047A1F1C04100F0AABA9EEA445FC8
:1098E00008D011EA5E0FBDE8104004BF01F000414E
:1098F00000207047BDE8104070B500F04BFA00BF83
:1099000064FBBE3E0000E0FF2DE9C04130B4DFF84B
:10991000A0C23CEA111418BF3CEA131400F0EC801A
:1099200081EA03051CEA111444EAD57418BF1CEA45
:10993000131500F0C780A4EB05044FF0004545EA7D
:10994000C12145EAC32341EA505143EA525304F18D
:109950007F74994204F500344FEAC0204FEAC222D6
:1099600008BF904200F09C804FEA13650FF240164A
:10997000765D4FEA134506FB05F7C7F1807706FBD6
:1099800007F74FEAD737A7FB03687642C8F5803858
:10999000A7FB06CE38BFA8F1010807FB08E64FF089
:1099A000000EA6FB028CE6FB03CEDCF1000CCEF130
:1099B000004E38BFAEF1010EA6FB0C584FF0000769
:1099C0004FF00005E6FB0E87A1FB08C6A0FB07CE03
:1099D00016EB0E0645F10005E1FB076515F1E04EBB
:1099E0007EBFA4F580345FEA46066D4116F180071C
:1099F00045F100054FEA17274FEA066647EA056773
:109A0000A6F1DE46B6F1805F4FEA15251FD938462C
:109A100024F0010C05EBC471BCF1FE6F01EB0C11DD
:109A200002D8F0BCBDE8008124425CBF01F5801E75
:109A30009EEAC47F02D4F0BCBDE80081244238D441
:109A4000F0BCA1F1C041BDE8004100F0F1B94FEA1E
:109A5000D22242EA43524FEAD323A7FB02864FEABF
:109A6000D02040EA415007FB03661EEA0E0F4FEA82
:109A7000D12105FB026658BFA6EB0056B6EB005697
:109A80004FEA520E4EEAC37E18EB0E0E56EB530E03
:109A9000BDD518EB02085E417F1C55F10005B6E705
:109AA0004FF480154FF000074FF000064FF000080C
:109AB000ADE7F0BC4FF0000001F1C04101F0004102
:109AC000BDE8008111EA0C1F0CEA131500D00CE070
:109AD00013EA0C1F00F025804FF00000F0BC81EA73
:109AE000030101F00041BDE80081F0BCBDE8004188
:109AF00081EA030100F09CB9F0BCBDE8004170B5FB
:109B000000F048F9097EFC3E00F007B881EA030145
:109B10004FF0000001F00041704781EA030100F0BE
:109B200087B9F0BCBDE800414FF000002149704703
:109B3000FFFDFBF9F7F5F4F2F0EEEDEBE9E8E6E412
:109B4000E3E1E0DEDDDBDAD8D7D5D4D3D1D0CFCD99
:109B5000CCCBCAC8C7C6C5C4C2C1C0BFBEBDBCBBD2
:109B6000BAB9B8B7B6B5B4B3B2B1B0AFAEADACABCD
:109B7000AAA9A8A8A7A6A5A4A3A3A2A1A09F9F9EA7
:109B80009D9C9C9B9A999998979796959594939359
:109B9000929191908F8F8E8E8D8C8C8B8B8A8989F0
:109BA0008888878786858584848383828281818073
:109BB0000000FF070000F87F4FEA1153A3F5806310
:109BC000D3F11E03A8BFD3F1200C08DB4FF00042F5
:109BD00042EAC12252EA505232FA03F07047094277
:109BE0000BD4102BC4BF0020704703F5787CBCF168
:109BF000FF3F05D04FF0FF3070474FF00000704737
:109C000070B500F0C7F800BF49922480002070476B
:109C1000F0E710F0004248BF4042B0FA80F310FA7B
:109C200003F10AD0C3F11D0303F580634FEA4150ED
:109C300002EB035202EBD12170474FF00000704756
:109C4000DFF848C170B51CEA111E1EBF1CEA1315CF
:109C50009EEA0C0F95EA0C0F00F06F8081EA030476
:109C600023EA4C134EEAD47E21EA4C1141F48011D0
:109C700043F48013AE44A1FB024CA0FB0365AEF19C
:109C80007F7E361955EB0C05A1FB034C4CF100030C
:109C9000A0FB021C16EB0C06654153F100030942C0
:109CA00018BF46F0010613F4007F0BD14FEA0331D1
:109CB0004FEA0530340341EA155140EA16506FF07F
:109CC00003020AE04FEAC3214FEAC520F40241EA49
:109CD000555140EA56506FF0020202EB2E4201EB62
:109CE000025585EACE710AD05FEA440C18BF24F011
:109CF000004450F1000041F1000120EAD47040F22C
:109D0000FE7C624500D270BDA84214BF4FF0804473
:109D10004FF04044002E08BF0024BEF1806FA8BF62
:109D2000A1F1C041BDE8704080F282804FF0000098
:109D300001F1C04101F0004170479EEA0C0F0CEAAE
:109D4000131518BF95EA0C0F06D04FF0000081EAFA
:109D5000030E0EF0004170BD00F01CF88900013EBA
:109D600000F007B800F009B84FEA430C5FEA5C5C0A
:109D700008D081EA030100F05BB84FEA410C5FEACA
:109D80005C5CF6D14FF00000014970470000FF070E
:109D90000000F87F0EF1020E2EF0030E5EF8046B49
:109DA000364205D4012A43EB030515F5001F12D8EE
:109DB000012841EB010C1CF5001F0CD80ED14FEA15
:109DC000D17C15F5001F0CEB4C0C0CF1020C08BFFC
:109DD0004CEBD37C04E04FF0080C01E04FEAD37C5D
:109DE0000CEB4C0526FA05F606F00706B6F1040C56
:109DF00006D20EEB860CBDE870404CF0010C6047BB
:109E0000DFE80CF0090B02024FF000414FF00000B8
:109E1000A1F5002170BD19461046012851EB01043F
:109E200018BFD4F5001484BF002001F0004170BDBC
:109E30000808A0F500114FEA3101704710B591EA0A
:109E4000030F48BF83F000433FF5BEAC841A71EBAB
:109E5000030C07D212198CF0004C43EB0C03001BCF
:109E600061EB0C01DFF8A4E14FEA1154A4EB135CA1
:109E70001EEA430F18BF9EEA445F00F0B08023EA59
:109E80006E03524221EA0451C3EB6E0338BF5B1EDE
:109E9000DCF1200E25D322FA0CFE10EB0E0043FA63
:109EA0000CFE41EB0E01CCF1200E03FA0EFE10EB7E
:109EB0000E0051F10001CCF1200E29D412FA0EF25D
:109EC00001EB0451BDE8104058BF7047401C1CBF57
:109ED000B2F1004F704700280CBF491C20F0010070
:109EE000704712EB020E43EB030218BF4FF0010E56
:109EF0004EEA4202ACF1200CDCF11E0E54D943FABA
:109F00000CFE10EB0E0051F1FF31CCF11E0ED5D539
:109F10000EF1010E12FA0EFE404141EB010101EB80
:109F2000445C5FEA5C5C10D910EBDE7001EB04511D
:109F300038BFBEF1004FBDE8104018BF7047002881
:109F40000CBF491C20F00100704730D24FEAD42CDE
:109F500011F5001124F400641BD0B1FA81F20B3A20
:109F6000A41AA41ED2F12003914030FA03F319433E
:109F7000904001EBCC71002C01EB0451BDE8104086
:109F8000A8BF704701F1C0414FF0000001F000414F
:109F90007047B0FA80F310FA03F100D110BDE41A53
:109FA000173C4805C90AE4E701EB045110BD49100C
:109FB00001EB0451BDE810404FEA300002E04FF0E1
:109FC000000170474A0008BF0042F8D0B2F5001FF8
:109FD00028BF704701F000414FF0000070479EEA33
:109FE000445F07D011EA5E0FBDE8104004BF0021B6
:109FF00000207047BDE8104070B5FFF7CBFE00BFF2
:10A0000040DFF63E83F00041104670470000E0FF5D
:10A010004FF04070E1EE100A7047FF2141EAD05046
:10A02000C00570470006101600061016000000005C
:10A0300000000000010203040607080900000000F8
:10A0400001020304240D25303123002B3030303041
:10A0500031002B3030303030002A2A005743535221
:10A06000303330303100524C5200574C5200524D78
:10A070004400525A5300575A53003031323334356A
:10A080003637383941424344454640305800303134
:10A09000323334353637383961626364656640304F
:10A0A0007800040000080000000000000002000129
:10A0B00000001000D4A000080000002014020000DE
:10A0C000C401000830A10008140200208420000010
:10A0D000200200080118729832104201035524F43E
:10A0E00013156D2A086013716E33080213A76F33BE
:10A0F00008031AB10832041A752032054BFD4D28A9
:10A10000011C692002B9C81AEE01A11DC0A872C2C3
:10A1100004156EFFFFFF1E546869732003000E577D
:10A1200066726F6D204348333935510D0A000000C7
:040000050800018965
:00000001FF
